:020000040800F2
:10000000E879002489040008BF7B00085F710008BC
:10001000BD7B0008AD08000849A8000800000000EA
:10002000000000000000000000000000C9030008FC
:100030001D0B00080000000025040008B780000820
:10004000A7040008A7040008A7040008A7040008E4
:10005000A7040008A7040008A7040008A7040008D4
:10006000A7040008A7040008A7040008F90800086E
:10007000A7040008A7040008A7040008A7040008B4
:10008000A7040008A7040008A7040008410B000803
:10009000590B00084D0B0008650B0008A704000869
:1000A000A7040008A7040008A7040008A704000884
:1000B000A7040008A7040008A7040008A704000874
:1000C000A7040008A7040008A7040008A704000864
:1000D000A7040008158D0008218D00082D8D00084B
:1000E000A7040008A704000800000000A7040008F7
:1000F000A7040008A7040008A7040008A704000834
:10010000A7040008A7040008A7040008A704000823
:10011000A7040008A7040008A7040008A704000813
:10012000A7040008A7040008A7040008A704000803
:10013000A7040008A7040008A7040008A7040008F3
:1001400000000000000000000000000000000000AF
:10015000A7040008A7040008A7040008A7040008D3
:10016000A7040008A7040008A7040008A7040008C3
:10017000A7040008E57C0008A704000800000000B0
:10018000A7040008A704000871860008A704000857
:10019000A7040008A7040008A7040008A704000893
:1001A000A7040008A7040008A70400080000000036
:1001B000A7040008A7040008A7040008A704000873
:1001C000A7040008A70400080000000000000000C9
:1001D0000000000000000000A7040008000000006C
:1001E000000000000000000000000000000000000F
:1001F0000000000000000000A7040008A704000899
:10020000A7040008A704000800000000A7040008D5
:10021000A7040008A7040008A7040008A704000812
:10022000A704000800000000A70400080000000068
:10023000A7040008A704000800000000A7040008A5
:10024000A7040008A7040008A7040008A7040008E2
:10025000A7040008A7040008A7040008A7040008D2
:10026000A7040008A7040008A7040008A7040008C2
:10027000A7040008A7040008A70400080000000065
:10028000A7040008A7040008A7040008A7040008A2
:1002900000000000A7040008A704000800000000F8
:1002A00000000000A7040008A7040008A704000835
:1002B000098D0008A7040008A7040008710B0008B6
:1002C0007D0B000851820008A704000800F002F826
:1002D00000F06AF80AA090E8000C82448344AAF176
:1002E0000107DA4501D100F05FF8AFF2090EBAE874
:1002F0000F0013F0010F18BFFB1A43F0010318475A
:1003000094BE0000D4BE00000A444FF0000C10F868
:10031000013B13F0070408BF10F8014B1D1108BF83
:1003200010F8015B641E05D010F8016B641E01F823
:10033000016BF9D113F0080F1EBF10F8014BAD1C73
:100340000C1B09D16D1E58BF01F801CBFAD505E091
:1003500014F8016B01F8016B6D1EF9D59142D6D3EB
:1003600070470000103A24BF78C878C1FAD8520705
:1003700024BF30C830C144BF04680C60704700001F
:100380000023002400250026103A28BF78C1FBD89E
:10039000520728BF30C148BF0B6070471FB50BF034
:1003A0008DFE1FBD10B510BD00F0D4F91146FFF74A
:1003B000F5FF0AF05BFA00F0F2F903B4FFF7F2FF81
:1003C00003BC00F0F9F900002C4B19680868B0E88C
:1003D000F04F80F30988BFF36F8F4FF0000080F378
:1003E000118870470000000008480068006880F32A
:1003F00008884FF0000080F3148862B661B6BFF33E
:100400004F8FBFF36F8F00DF00BF00BF08ED00E02C
:10041000DFF80C00016841F470010160704700BF13
:1004200088ED00E0EFF30980BFF36F8F134B1A687C
:100430001EF0100F08BF20ED108A20E9F04F106069
:1004400009B44FF0500080F31188BFF34F8FBFF312
:100450006F8F0BF0FDF84FF0000080F3118809BC9E
:1004600019680868B0E8F04F1EF0100F08BFB0EC34
:10047000108A80F30988BFF36F8F70474C00002407
:10048000EFF30580704700000A4880470A4880471C
:100490000A480047FEE7FEE7FEE7FEE7FEE7FEE765
:1004A000FEE7FEE7FEE7FEE705480649064A074B7A
:1004B00070470000250B000879810008CD02000874
:1004C000E8190024E8790024E8390024E8390024F8
:1004D00053EA020C00F069802DE9F04B4FF0000662
:1004E000002B1FBFB3FA83F503FA05F424FA05F6CF
:1004F0005E4012BF1643B2FA82F502FA05F4C5F166
:1005000020051EBF22FA05FC44EA0C04203556EAF9
:10051000044C4FEA144418BF641C4FF000084FF01D
:100520000009904271EB030C39D3002919BFB1FACD
:1005300081F701FA07F6B0FA80F700FA07F6C7F17B
:1005400020071EBF20FA07FC46EA0C062037B6FB40
:10055000F4FCA7EB0507103F07F01F0BCBF12006BB
:100560000CFA0BFB2CFA06F644BFB3460026202FEC
:10057000A4BF5E464FF0000B5BEA060C08BF4FF0CD
:10058000010B19EB0B09ABFB027C48EB0608C01B07
:1005900006FB02CC0BFB03CC71EB0C01C1E70B4655
:1005A000024641464846BDE8F08B13B54FF00000C7
:1005B0004FF00001AFF30080BDE81C407047032AF4
:1005C00040F2308010F0030C00F0158011F8013B70
:1005D000BCF1020F624498BF11F801CB00F8013B57
:1005E00038BF11F8013BA2F1040298BF00F801CB1B
:1005F00038BF00F8013B11F0030300F02580083AF2
:10060000C0F0088051F8043B083A51F804CBA0E848
:100610000810F5E7121D5CBF51F8043B40F8043B9D
:10062000AFF30080D20724BF11F8013B11F801CBD2
:1006300048BF11F8012B24BF00F8013B00F801CBA3
:1006400048BF00F8012B704710B5203AC0F00B806E
:10065000B1E81850203AA0E81850B1E81850A0E8C6
:100660001850BFF4F5AF5FEA027C24BFB1E8185020
:10067000A0E8185044BF18C918C0BDE810405FEA90
:10068000827C24BF51F8043B40F8043B08BF70470C
:10069000D20728BF31F8023B48BF11F8012B28BF11
:1006A00020F8023B48BF00F8012B704702F0FF031F
:1006B00043EA032242EA024200F02CB84FF0000263
:1006C00000B5134694469646203922BFA0E80C5048
:1006D000A0E80C50B1F12001BFF4F7AF090728BF23
:1006E000A0E80C5048BF0CC05DF804EB890028BF9F
:1006F00040F8042B08BF704748BF20F8022B11F0C8
:10070000804F18BF00F8012B704770477047704743
:100710004FF000020429C0F0128010F0030C3FF4E7
:10072000CFAFCCF1040CBCF1020F18BF00F8012BC5
:10073000A8BF20F8022BA1EB0C01FFF7C1BF5FEAB5
:10074000C17C24BF00F8012B00F8012B48BF00F842
:10075000012B7047754600F02BF8AE460500694640
:10076000534620F00700854618B020B5FFF79CFEE1
:10077000BDE820404FF000064FF000074FF00008A2
:100780004FF0000B21F00701AC46ACE8C009ACE823
:10079000C009ACE8C009ACE8C0098D46704710B587
:1007A0000446AFF300802046BDE81040FFF705BEC9
:1007B000004870478819002401491820ABBEFEE7A5
:1007C000260002007047000010B532490446006858
:1007D000884202D0304A904202D1D1F8080302E0A8
:1007E0002E48D0F8080310F4403F10D004F0FCFF6E
:1007F0006168B1F5803F06D0B1F5003F03D0B1F597
:10080000403F26D101E0090C17E0800821E00021DB
:100810004FF4002004F0A0F861688A03920B18D10D
:100820008A140C2A15D2DFE802F014060606060622
:10083000060B0D0F1113890C4900B0FBF1F008E015
:10084000000906E0400904E0800902E0C00900E078
:10085000000A13494008884204D82068816821F4BE
:10086000407108E00F49884207D82068816821F468
:10087000407141F48071816010BD0B49884220684D
:10088000816804D821F4407141F40071F3E741F428
:100890004071F0E700200240002102400060025851
:1008A000105E5F0020BCBE0040787D01FEE70020A6
:1008B000704700207047000005490022054810B528
:1008C00008F020FC0449034808F00FFC002010BD8C
:1008D000E8110020D4020024E80900200146044861
:1008E00010B508F002FC024808F0D8FB002010BD4B
:1008F000D402002400207047014801F097BA00009C
:1009000030010020294A016891423AD0274A183222
:10091000914236D0254A3032914232D0234A483271
:1009200091422ED0214A603291422AD01F4A783219
:10093000914226D01D4A9032914222D01B4AA832C1
:1009400091421ED01A4A91421BD0194A1832914244
:1009500017D0174A3032914213D0154A483291428B
:100960000FD0134A603291420BD0114A7832914233
:1009700007D00F4A9032914203D00D4AA8329142DB
:1009800011D1CAB21823103AB2FBF3F26FF3090186
:10099000032A02F00703074AD25CC26500D9091D89
:1009A00081650846704721F0FF01F9E71000024019
:1009B00010040240ECC0000830B5224A012301684F
:1009C0009142CAB21BD01F4C1434A14217D01D4C07
:1009D0002834A14213D01B4C3C34A1420FD0194CF7
:1009E0005034A1420BD0174C6434A14207D0154CAF
:1009F0007834A14203D0134C8C34A1420CD1142181
:100A0000114C083AB2FBF1F10F4A803201F01F0598
:100A100004EB8101AB4010E00C4D1824103A0D445A
:100A2000B2FBF4F1A82D00D80831094A01F01F04E7
:100A300002EB8101064AA3408032603080E80E005C
:100A400030BD00000854025800580258F0FBFDBFAA
:100A50000008024010B50279531E072B2DD8174C01
:100A60000168A1421BD0154C1434A14217D0134C7D
:100A70002834A14213D0114C3C34A1420FD00F4C6A
:100A80005034A1420BD00D4C6434A14207D00B4C22
:100A90007834A14203D0094C8C34A14203D10849D7
:100AA000074C443102E00749064C443104EB820212
:100AB000C0E91B2101219940416710BD085402582B
:100AC000FC580258FC08024010B583694FF0C0740E
:100AD000826A0146002053B1B3F5005F15D072B1B0
:100AE000012A0CD0022A0AD0032A09D104E01AB143
:100AF000012A06D0022A03D1C96AC90100D5012002
:100B000010BDC96AA142FAD010BD002AF7D0012A4F
:100B1000F2D0022AF3D0032AF3D010BD704772B688
:100B2000FEE70000054805490839026842F0020264
:100B3000026008688004FCD5704700000C48025829
:100B4000014801F0DBBE0000A8010020014801F0CF
:100B5000D5BE0000A8010020014801F0CFBE000072
:100B600048020020014801F0C9BE000048020020F0
:100B7000014801F0C3BE0000E8020020014801F076
:100B8000BDBE0000E8020020F0B503684FF6FC711E
:100B90006D4C426BD3F884508D4345EA8205C3F80F
:100BA0008450036853F8845F068F25F47F0545EA77
:100BB00006451D60836B654D9F180268D2F888302A
:100BC0008B4343EA8703C2F88830026852F8883FB3
:100BD000868F23F4FE0343EA06431360066856F843
:100BE000A03FC26B8B4307EB420243EA82033360B0
:100BF000076857F8A03FB0F8406023F4FE0343EACB
:100C000006433B60D0E9103603FB06220368D3F8A5
:100C1000B0608E4346EA8206C3F8B0600368B0F85D
:100C20004860D3F8B07027F4FE0747EA0646C3F8D9
:100C3000B060D0E91267036806FB0722D3F8AC6006
:100C40008E4346EA8206C3F8AC60D0E914670368B5
:100C500006FB0722D3F8F0608E4346EA8206C3F80B
:100C6000F0600368B0F85860D3F8F07027F47C1790
:100C700047EA0646C3F8F0600368876D53F8C06F13
:100C800002EB47028E4346EA820119600168B0F820
:100C90005C20D1F8C03023F47C1343EA0242C1F84F
:100CA000C020016890F86020D1F8C03023F07C5358
:100CB00043EA0262C1F8C020416B04EB8101C166C6
:100CC000826B01EB82020267C36B02EBC3024267D5
:100CD000D0E91034634302EB83028267D0E9123417
:100CE000634302EB8302C267D0E91434634302EB2F
:100CF0008302C0F88020836D02EBC303C0F8843008
:100D0000C46D826E544303EB8403C0F88830046ED4
:100D1000544303EB8402C0F89020AA420AD9D0F8C9
:100D20009C20032142F02002C0F89C2080F89810FB
:100D30000120F0BD002200E004C1D0F890308B42C9
:100D4000FAD80020F0BD000000AC0040FCD3004009
:100D50002DE9F0470F4690F85C109CB0044601293D
:100D60004FF0000915D00026DFF8F880012084F844
:100D70005C0018961996216841450ED13A4D0095B0
:100D8000284606F017FA8246206806F013FA60B18A
:100D90000EE002201CB0BDE8F087206E84F85C6095
:100DA00040F0200020660120F4E7BAF1000F09D0DE
:100DB000216E4FF0010941F020002066484684F87A
:100DC0005C60E7E720684146884201D0A84201D133
:100DD000264800E0264840F61F72D7F800C0254B91
:100DE000BCF1000F23D0D0F808C0D7F804802CF451
:100DF000404C4CEA080CC0F808C0D4F800C08C4540
:100E000001D0AC4507D18968AB6801F0010103F05E
:100E10000103194302E0996801F001010029CDD1D5
:100E2000BD683968836829439343194317E087688D
:100E300027F44047876027688F4201D0AF4207D12F
:100E40008968AB6801F0010103F00103194302E076
:100E5000996801F001010029B0D181689143816056
:100E6000ACE70000002002400021024000230240C5
:100E700000630258006002582DE9F84F0446DFF87D
:100E8000ECB30020FA4E0090814694F85C000D46C9
:100E9000F84F012808D04FF0010A84F85CA02068C0
:100EA00006F084F918B18FE20220BDE8F88F2868B7
:100EB00000280FDB2168B1420CD0CA69030327D098
:100EC00090FAA0F0B0FA80F000F01F030AFA03F0E5
:100ED0000243CA61D5E900124FF00C0C20681F23B1
:100EE000C1F384610CEA921C02F01F02604493403B
:100EF0009140026B9A430A430263206806F056F958
:100F00008046206806F04EF958EA000003D054E10C
:100F1000C0F38460D8E729684FF0040C20680723E9
:100F2000AA680CEAD15CC1F3045160448B408A404A
:100F300041699943114341612068B04204D1C268BC
:100F40006969C2F3C1020BE0CB4A1268BAEB127FA7
:100F500002D0C168C90605D4C2686969C2F38202B9
:100F6000520004E0C268696902F010025208914020
:100F70002A69042A5AD02B6800EB8202B04202F19F
:100F8000600207D103F0F8401368084340F00040C6
:100F9000106008E0D2F800C003F0F84008430CF0FD
:100FA0000041014311602068B0421CD12969EA69FF
:100FB00000EB8100016E21F080711143016695F80C
:100FC000201020682A6901290AD00021B0429ED150
:100FD00000EB8200026E22F000720A430266ECE02F
:100FE0004FF00071F2E795F821102A69012917D016
:100FF0005FF0000100EB8200026E22F000420A4323
:101000000266297E20682A6901290CD00021036923
:1010100002F01F02914023F4F0420A430261CCE047
:101020004FF00041E6E74FF40061F0E7B04273D1C2
:10103000002106F0B1F8000320684FF000016DD0E8
:1010400006F0AAF890FAA0F0B0FA80F1286802033E
:1010500069D090FAA0F0B0FA80F0814204D1002269
:101060002068114606F0AAF82068012106F094F8DD
:10107000000320684FF0010158D006F08DF890FA77
:10108000A0F0B0FA80F12868020354D090FAA0F0E2
:10109000B0FA80F0814204D120680022012106F0DC
:1010A0008DF82068022106F077F8000320684FF0E1
:1010B000020143D006F070F890FAA0F0B0FA80F187
:1010C000286802033FD090FAA0F0B0FA80F0814285
:1010D00004D120680022022106F070F82068032164
:1010E00006F05AF8000320684FF003012ED006F0F6
:1010F00053F890FAA0F0B0FA80F1286802032AD0E1
:1011000090FAA0F0B0FA80F0814256D12068002217
:10111000032106F053F850E020E0FFE706F03CF82A
:10112000C0F3846192E7C0F3846096E706F034F878
:10113000C0F38461A7E7C0F38460ABE706F02CF846
:10114000C0F38461BCE7C0F38460C0E706F024F814
:10115000C0F38461D1E7C0F38460D5E7016E2A78DB
:1011600001F0F841B1EB826F03D1016E21F0004133
:10117000016620682978426E02F0F842B2EB816F76
:1011800003D1416E21F00041416620682978826ECA
:1011900002F0F842B2EB816F03D1816E21F0004181
:1011A000816620682978C26E02F0F842B2EB816F46
:1011B00003D1C16E21F00041C1662068816811F041
:1011C000010F52D12D4AB042EB6829680FD1D0F8F7
:1011D000B0C003F01808C1F3130322FA08F20A4062
:1011E0002CEA030C4CEA020CC0F8B0C00EE0D0F8B8
:1011F000C0C003F01808C1F3130322FA08F20A4032
:101200002CEA030C4CEA020CC0F8C0C0E96859454E
:1012100070D11B482268DFF86CC0DFF86CB08242E6
:10122000DFF868E01A481B4BDFF86C8043D129686F
:10123000614565D0B1EB4C0C6DD0714569D0A1F121
:10124000865CBCF1100C75D0DFF850C061456DD0E4
:10125000DFF84CC061457FD0814273D0994247D0BE
:101260001048814222D1104876E0B3E00000FF47E9
:1012700000600258002102400010005CFFFF0F00D8
:101280000020024002003004400020190800900CA9
:101290000008302E00106032002090362000F0143C
:1012A0000004002A00002143000052476E4881429A
:1012B00051D16E4850E0BA421DD1296861451FD016
:1012C000A1F1066CBCF1040C25D0714521D0A1F12F
:1012D000865CBCF1100C2DD0DFF894C1614525D09F
:1012E000DFF890C1614537D081422BD09942DDD1E2
:1012F000404631E040E0B2422DD12968614501D13C
:10130000012029E0A1F1066CBCF1040C03D0714569
:1013100003D1594820E058461EE0A1F1865CBCF19B
:10132000100C07D0DFF848C1614505D1534813E0E0
:1013300000E007E052480FE0DFF838C161450BD00C
:10134000814201D1184607E04E48414504D0814210
:1013500001D14D4800E00020B2420DD0D169030315
:101360001AD090FAA0F0B0FA80F000BF00F01F038E
:101370000AFA03F00143D161D5F800C0BCF1000FB7
:1013800028DA424B20684249DFF808A1984201D090
:10139000B84203D10A4602E0800EE7E7524692685F
:1013A000984202F0E07201D0B84209D19D68D7F8A6
:1013B000088005F0010508F0010845EA080502E08B
:1013C000B56805F0010555B1216E4FF0010941F0F6
:1013D00020002066002084F85C00484665E52E4D1C
:1013E000AC451CD115021AD4B042F3D1984202D0B8
:1013F000B84200D051468B6842F4000023F0E072FE
:1014000002438A60264925480968B1FBF0F0400094
:10141000801C00E0401E00900028FBD1DAE7214D3F
:10142000AC450CD1D5010AD4B042D3D1984202D0F8
:10143000B84200D051468B6842F080700EE01A4DE1
:10144000AC45C7D15502C5D4B042C3D1984202D0F1
:10145000B84200D051468B6842F4800023F0E0721D
:1014600002438A60B6E700000000844B0000B84FDA
:101470002000F0140004002A8000501D0002B02556
:10148000000180210040C03A0080F03E0020024070
:101490000023024000630258000052C7400D0300C1
:1014A00044000024000021C3000084CB2DE9F84350
:1014B0004FF0000504002E46009502D0206E18B1B2
:1014C00008E00120BDE8F883204600F043F9656696
:1014D00084F85C5020688168C1F3407119B181685B
:1014E0008E4A1140816020688168C1F3007181B922
:1014F00081688B4A114041F0805181608A49894856
:101500000968B1FBF0F0401C00E0401E009000288C
:10151000FBD120688168C1F3007141B9216E0126B9
:1015200041F010012166616E41F00101616605F034
:101530003DFE216EC90600D420B1206E012640F088
:101540001000E0E0206E20F4807040F00200206681
:1015500020688168754D11F0010F1ED1744B754ADA
:10156000984201D0904207D19968976801F0010133
:1015700007F00107394302E0A96801F0010161B9F0
:10158000984201D0904201D16B4800E06B488268DC
:10159000616822F47C120A4382602168A9421FD14B
:1015A000637ED4E90207E26B5B033A43082805D067
:1015B0000C280FD01C280FD018280FD05FF0000087
:1015C00000F00C0794F8200043EA47031A4342EA6C
:1015D00000400FE00420F3E70820F1E71C20EFE7CC
:1015E000627E94F82030A768E06B520342EA03421F
:1015F0003843104394F82020012A04D1A28C504B88
:1016000003EB42421043A26A2AB1E36A02F4787201
:10161000024343EA0200CA68A9420BD1494B1A406F
:101620000243CA602068626B016921F04061114386
:10163000016103E0444B1A400243CA60206805F090
:10164000B5FD0746206805F0ADFD07434ED1206883
:10165000A946484506D1217E94F83820890341EAFD
:10166000420103E0227E216B41EA8231C26844F2EA
:1016700003039A430A43C26094F844000128206897
:1016800003D0016921F0010122E048450ED1D4E9DF
:10169000121CD4E9143502692C4F41EA0C012B438A
:1016A0003A401943114341F0010111E0D4E9131705
:1016B000B4F848C0DFF89880636D026908EB0C4C01
:1016C000224D394343EA0C036D1E2A40194311434E
:1016D00001612068236C026922F070421A430261A2
:1016E0002068484502D02046FFF76EF8206901289F
:1016F00020680BD0016B21F00F010163206E20F0F8
:10170000020040F0010020663046DBE6E269016B32
:10171000521E21F00F011143EFE70000C0FFFF5FF1
:10172000C0FFFF7F400D030044000024006002580A
:1017300000200240002102400023024000630258C2
:101740000000FEFF0740F0FF03C0F0FF1FF800FCA1
:101750000100FFFFF0B5B5B0064614212EA8FEF734
:10176000ADFFB8216846FEF7A9FF314930688842CD
:101770005BD1022000224FF400210091CDE901202D
:101780001024154606AACDE90340C023059082E83F
:10179000290068460995289503F02CFA08B1FFF74F
:1017A000BEF92448016841F020010160006800F0A2
:1017B000200033901F480830016841F001010160AA
:1017C000016801F001013391016841F004010160F9
:1017D000006803272EA9309500F0040033902020E4
:1017E000CDE92E07144801F02FFC14482EA9CDE9AD
:1017F0002E47309501F028FC114C092111484FF477
:10180000807C021584E82300D700C4E90352C31486
:101810002046C4E907C56562C4E9053700F07AFED1
:1018200008B1FFF77CF9B465A66335B0F0BD0000E0
:1018300000200240D8440258000002580008025814
:1018400030010020100002402DE9F84F044601F05D
:101850000FFD00903CB194F83500022806D080219D
:1018600061650020E4E00120BDE8F88FC74DC74E58
:10187000C649183520683036DFF81483DFF8149332
:101880008842DFF814A3DFF814B32ED0A8422CD07E
:10189000B0422AD0404528D0484526D0504524D0D3
:1018A000584522D0BD4A183290421ED0BC4A9042C0
:1018B0001BD0BB4A1832904217D0B94A30329042FE
:1018C00013D0B74A483290420FD0B54A60329042A6
:1018D0000BD0B34A7832904207D0B14A903290424E
:1018E00003D0AF4AA832904209D1026822F01E020A
:1018F00002602068426922F08002426103E00268CF
:1019000022F00E02026027688F4238464DD0A8426E
:101910004BD0B04249D0404547D0484545D05045CE
:1019200043D0584541D09D4A183290423DD09C4A00
:1019300090423AD09A4A1832904236D0984A303281
:10194000904232D0964A483290422ED0944A603229
:1019500090422AD0924A7832904226D0904A9032D1
:10196000904222D08E4AA83290421ED08D4A904298
:101970001BD08C4A1432904217D08A4A28329042A7
:1019800013D0884A3C3290420FD0864A503290425F
:101990000BD0844A6432904207D0824A7832904217
:1019A00003D0804A8C32974204D1206E026822F420
:1019B0008072026075492068884228D0A84226D0EB
:1019C000B04224D0404522D0484520D050451ED0BA
:1019D00058451CD071491831884218D07049884246
:1019E00015D06F491831884211D06D493031884285
:1019F0000DD06B494831884209D06949603188422D
:101A000005D067497831884201D065499031016835
:101A100021F0010101600EE001F02AFC0099401A5A
:101A2000052808D9202262650321002084F835109A
:101A300084F8340017E73868C007EDD1534A012114
:101A4000206890422ED0A8422CD0B0422AD04045E7
:101A500028D0484526D0504524D0584522D04F4B59
:101A6000183398421ED04E4B98421BD04C4B183323
:101A7000984217D04A4B3033984213D0484B4833E2
:101A800098420FD0464B603398420BD0444B78338A
:101A9000984207D0424B9033984203D0404BA83332
:101AA000984208D194F85C703F23A06D07F01F079F
:101AB000BB40836007E094F85C30A06D03F01F0327
:101AC00001FA03F34360206890424DD0A8424BD006
:101AD000B04249D0404547D0484545D0504543D015
:101AE000584541D02D4A183290423DD02C4A904260
:101AF0003AD02B4A1832904236D0294A303290429E
:101B000032D0274A483290422ED0254A6032904245
:101B10002AD0234A7832904226D0214A90329042ED
:101B200022D01F4AA83290421ED01E4A90421BD09B
:101B30001C4A1432904217D01A4A2832904213D0CD
:101B4000184A3C3290420FD0164A503290420BD085
:101B5000144A6432904207D0124A7832904203D03D
:101B6000104A8C3290420BD1D4E919024260E06EE7
:101B700030B1026822F480720260D4E91C02426033
:101B8000002084F8351084F834006DE6100002401F
:101B9000580002407000024088000240A00002404D
:101BA00010040240085402582DE9F05F28B190F863
:101BB0003510022904D0802141650120BDE8F09F45
:101BC000904C904B0168183C18338E4ADFF83C92D9
:101BD000A1428D4CDFF838E28E4FDFF83CB2DFF8DF
:101BE0003CA28F4D8F4E31D091422FD099422DD0B3
:101BF000A1422BD0494529D0714527D0B94225D0E3
:101C0000DFF810C20CF1180C61451FD0DFF808C2D4
:101C1000ACF1600C614519D0DFF8FCC1ACF1480CA7
:101C2000614513D0DFF8F0C1ACF1300C61450DD047
:101C3000DFF8E4C1ACF1180C614507D0594505D077
:101C4000514503D0A94201D0B1422CD1DFF8B4C133
:101C50004FF0040880F83580ACF1180C61451DD0B8
:101C600091421BD0994219D0A14217D0494515D0B5
:101C7000714513D0B94211D06648183081420DD059
:101C800065486038814209D063484838814205D0B0
:101C900061483038814201D05F481838086820F028
:101CA00001000860ABE0D1F800C02CF00E08DFF8AE
:101CB00054C1C1F80080ACF1180C0168614527D00F
:101CC000914225D0994223D0A14221D049451FD02D
:101CD00071451DD0B9421BD0DFF838C10CF1180C8A
:101CE000614515D0DFF830C1ACF1600C61450FD013
:101CF000DFF824C1ACF1480C614509D0DFF818C108
:101D0000ACF1300C614503D0DFF80CC1ACF1180C1C
:101D1000D1F800C02CF0010CC1F800C0DFF8E4805D
:101D20004FF0010C0168A8F11808414546D09142D6
:101D300044D0994242D0A14240D049453ED071455D
:101D40003CD0B9423AD0334A1832914236D0324A66
:101D5000603A914232D0304A483A91422ED02E4ACF
:101D6000303A91422AD02C4A183A914226D059450D
:101D700024D0514522D0A94220D0B1421ED02A4AB7
:101D800091421BD0284A1432914217D0264A283259
:101D9000914213D0244A3C3291420FD0224A503211
:101DA00091420BD0204A6432914207D01E4A7832C9
:101DB000914203D01C4A8C32914218D1016E0A68BC
:101DC00022F480720A6090F85C20816D02F01F029C
:101DD0000CFA02F24A60D0E919124A60C16E31B1C0
:101DE0000A6822F480720A60D0E91C124A6000225C
:101DF000016D80F835C080F8342001B1884700209B
:101E0000DCE600002800024058000240700002405A
:101E100088000240A0000240700402408804024092
:101E2000A0040240B8040240085402582DE9FC5FA7
:101E30000446F74E0020DFF8D88300904FF4165286
:101E4000F44808F11808A56DDFF8C493DFF8C0A3C3
:101E5000016809F1300920680AF1480AB1FBF2F182
:101E6000B04201912F68D5F800C0DFF8ACB335D08F
:101E70004146884232D0484530D050452ED0584552
:101E80002CD0E5491831884228D0E34930318842C6
:101E900024D0E1494831884220D0E04988421DD011
:101EA000DE491831884219D0DC493031884215D0DA
:101EB000DA494831884211D0DFF860E30EF1600E54
:101EC00070450BD0D54A7832904207D0D34B90332F
:101ED000984203D0D149A83188427DD194F85C2042
:101EE000082102F01F0201FA02F23A424AD0B0423F
:101EF00032D0404530D048452ED050452CD05845A2
:101F00002AD0C54A1832904226D0C34A3032904275
:101F100022D0C14A483290421ED0C04A90421BD0C3
:101F2000BE4A1832904217D0BC4A3032904213D089
:101F3000BA4A483290420FD0B84A603290420BD031
:101F4000B64A7832904207D0B44A9032904203D0D9
:101F5000B24AA832904203D1026802F0040202E0C1
:101F6000026802F008026AB1026822F0040202600C
:101F700094F85C0000F01F008140A960606D40F0A3
:101F80000100606594F85C00012100F01F008140B1
:101F9000394240D02068B04234D0404532D0484524
:101FA00030D050452ED058452CD09B4A1832904204
:101FB00028D0994A3032904224D0974A48329042F1
:101FC00020D0964A90421DD0944A1832904219D09F
:101FD000924A3032904200E0AFE113D08F4A48324B
:101FE00090420FD08D4A603290420BD08B4A7832AB
:101FF000904207D0894A9032904203D0874AA83253
:1020000090427DD1406910F0800F04D0A960606DCE
:1020100040F00200606594F85C00042100F01F00AD
:10202000814039423ED02068B04232D0404530D065
:1020300048452ED050452CD058452AD0764A1832E3
:10204000904226D0744A3032904222D0724A4832AE
:1020500090421ED0714A90421BD0704A1832904272
:1020600017D06E4A3032904213D06C4A48329042B8
:102070000FD06A4A603290420BD0684A7832904260
:1020800007D0664A9032904203D0644AA832904208
:102090004ED1006810F0020F04D0A960606D40F0CE
:1020A0000400606594F85C00102100F01F0081407E
:1020B000394258D02068B04234D0404532D04845EB
:1020C00030D050452ED058452CD0534A183290422B
:1020D00028D0514A3032904224D04F4A4832904260
:1020E00020D04E4A90421DD04C4A1832904219D00E
:1020F0004A4A3032904215D0484A4832904200E075
:1021000014E00FD0454A603290420BD0434A7832F7
:10211000904207D0414A9032904203D03F4AA832C1
:10212000904207D1006800F0080006E0006872E7FE
:102130000068B7E7006800F00400A0B1A96020685B
:102140000168490304D50068000308D5A16C07E0C5
:102150000168C90503D4016821F008010160216C00
:1021600009B12046884794F85C00202100F01F0048
:102170008140394279D02068B04232D0404530D0D9
:1021800048452ED050452CD058452AD0224A1832E6
:10219000904226D0204A3032904222D01E4A483205
:1021A00090421ED01D4A90421BD01C4A18329042C9
:1021B00017D01A4A3032904213D0184A483290420F
:1021C0000FD0164A603290420BD0144A78329042B7
:1021D00007D0124A9032904203D0104AA83290425F
:1021E00003D1006800F0100002E0006800F0020077
:1021F000B0B3A96094F835000428206801680FD0B6
:1022000049037ED5006800032BD4616C2AE00000EE
:1022100010000240440000247000024010040240FC
:1022200021F0160101602068416921F080014161BF
:10223000206C08B9A06C20B12068016821F0080169
:10224000016094F85C303F21012003F01F0300225D
:102250009940A96084F8350084F83420216D65E048
:1022600003E0E16B09B120468847606D00287DD00E
:10227000606DC00759D02068042184F83510B04241
:102280002BD0404529D0484527D0504525D058452A
:1022900023D09D49884220D09B49183188421CD0C8
:1022A00099493031884218D09849884215D09749C9
:1022B0001831884211D09549303188420DD0934968
:1022C0004831884209D091496031884205D08F4910
:1022D0007831884201D08D499031016821F00101A7
:1022E000016020680099019A491C0091914202D82E
:1022F0000168C907F6D10068C00710D003200FE0BD
:10230000FFE70168C905ACD403680121002223F06E
:102310001003036084F8351084F83420A1E701200D
:1023200084F83500002084F83400E16C00291DD0C9
:1023300002B02046BDE8F05F0847754988421DD0CD
:1023400073491431884219D071492831884215D017
:102350006F493C31884211D06D49503188420DD0CF
:102360006B496431884209D0694900E084E07831E2
:10237000884203D066498C3188427DD194F85C80D4
:102380000427016808F01F0807FA08F717EA0C0F7E
:10239000009746D04F0744D500980F04686003D5D6
:1023A000C8033CD4A16CC1E7880638D42068B04289
:1023B0002DD055496039884229D0484527D050450D
:1023C00025D0584523D05049884220D04E49183155
:1023D00088421CD04C493031884218D04B49884241
:1023E00015D04A491831884211D0484930318842C5
:1023F0000DD046494831884209D0704507D09042F7
:1024000005D0984203D04149A831884203D10168E0
:1024100021F0080102E0016821F004010160216C53
:1024200084E7022707FA08F717EA0C0F00974ED047
:102430008F074CD500980F04686003D5C80344D4B7
:10244000616C73E7880640D42068B0422FD02E49D3
:10245000603988422BD0484529D0504527D058456F
:1024600025D02949884222D02749183188421ED0D8
:1024700025493031884200E044E018D023498842A1
:1024800015D022491831884211D020493031884274
:102490000DD01E494831884209D0704507D090427E
:1024A00005D0984203D01949A831884203D1016868
:1024B00021F0140102E0016821F00A01016001210C
:1024C00084F83510002084F83400E16B2EE70822F0
:1024D00002FA08F212EA0C0F14D0090712D50168AB
:1024E00021F00E01016094F85C100120002201F03F
:1024F0001F0100FA01F16960606584F8350084F815
:10250000342012E7BDE8FC9F88000240100402401E
:10251000085402582DE9F05F044600F0A9FE002C93
:1025200007467DD0E24E022120684FF00308DFF815
:1025300084934FF00005DFF880A3B042DFF87CB34E
:1025400034D0DB4A1832904230D048452ED0504526
:102550002CD058452AD0D94A1832904226D0D74A92
:102560003032904222D0D54A483290421ED0D44ACE
:1025700090421BD0D24A1832904217D0D04A303203
:10258000904213D0CE4A483290420FD0CC4A6032AB
:1025900090420BD0CA4A7832904207D0C84A903253
:1025A000904203D0C64AA83290427DD184F83510BB
:1025B000B04284F834502ED0BD49183188422AD018
:1025C000484528D0504526D0584524D0BB4918311D
:1025D000884220D0B949303188421CD0B7494831AF
:1025E000884218D0B649884215D0B549183188427A
:1025F00011D0B349303188420DD0B14948318842B9
:1026000009D0AF496031884205D0AD497831884260
:1026100001D0AB499031016821F00101016008E06F
:1026200025E100BF00F024FEC01B052801D92021B0
:102630001AE120680068C007F4D1D4E902032168D8
:10264000103418438E4694E88410D4E9033809689E
:102650003A4310439B4A40EA0C0067691843114013
:10266000103C40EA0800042F40EA010003D1D4E9FD
:102670000B12114308436168A1F12902052A0BD905
:10268000163A032A08D9083A012A05D9083A032A32
:1026900002D97439032901D840F48010CEF8000023
:1026A0002068676A406900E020E0042F20F00700FE
:1026B00047EA00070DD1D4E90A01074349B1204692
:1026C000FEF702FA28B140206065012184F8351038
:1026D000CDE0206847612046FEF714F994F85C20AD
:1026E0003F2102F01F029140816055E0764A9042FE
:1026F0001BD0754B1433984217D0734B2833984234
:1027000013D0714B3C3398420FD06F4B50339842EB
:102710000BD06D4B6433984207D06B4B78339842A3
:1027200003D0694B8C3398427ED184F8351084F8FD
:102730003450664B0168A26801EA030E402A74D047
:10274000802A73D05FF00002D4E90378D4E9053120
:1027500042EAD70242EAD8085B4AD4E9077C48EA51
:10276000D30848EAD10141EAD701524241EA1C119B
:10277000142341EA0E01016020681044B0FBF3F01D
:102780008000E0652046FEF7BDF894F85C2001214A
:1027900002F01F02914041602068B04257D0444986
:1027A0001831884253D0484551D050454FD05845F4
:1027B0004DD042491831884249D040493031884291
:1027C00045D03E494831884241D03D4988423ED0BB
:1027D0003B49183188423AD039493031884236D0A5
:1027E00037494831884232D03549603188422ED04D
:1027F0003349783188422AD031499031884226D0F5
:102800002F49A831884222D02F4988421FD02E4913
:10281000143188421BD02C492831884217D02A49CC
:102820003C31884213D002E01DE017E018E0264951
:10283000503188420BD024496431884207D0224964
:102840007831884203D020498C31884229D12046F2
:10285000FEF7B2F8A06880280CD00CE0102273E7D5
:102860004FF4804270E74021616584F83580012093
:10287000BDE8F09F6560216E20790860D4E91901F8
:1028800041606068401E072808D82046FEF7E2F83D
:10289000E06E0560D4E91C01416002E0E566256751
:1028A00065670120656584F835000020E0E70000D9
:1028B00010000240400002405800024070000240F8
:1028C000100402403F8010FE085402580F00FEFF23
:1028D00070B5044600F0CCFC0546601C02D00448EC
:1028E0000078044400F0C4FC401BA042FAD370BD41
:1028F0003800002470477047704770472DE9FF5F2C
:10290000DFF80CB304460BF10401DBF80000256886
:102910000F68AA468007D5F85090696DD5F85080A9
:102920006E6D2A6DD5F854C02B6D00EA877000904B
:1029300009F470496F6D286D01EA09010191DAF817
:102940005410DAF85490DAF8505008F00F0806EAFC
:102950000806029602F0F00203F071536FEA0906CE
:102960001F4000F060700CEA020CCDF80CC0F205BC
:1029700001EA00090CD4E843C00509D400214FF452
:102980008073CAF85030CBF800102046FFF7B5FF2F
:10299000700512D4E84340050FD4206800234FF49B
:1029A0008068D0F8DC20D0F8E410C0F85080CBF874
:1029B00000301140204600F042FBDFF858A200989A
:1029C00050B12268830F00EA0A001065CBF800308E
:1029D00020460099FFF78EFF019850B12268830FBF
:1029E00000EA0A001065CBF800302046019900F09B
:1029F00028FB029850B12268830F00EA0A00106594
:102A0000CBF800302046029900F011FB039850B13A
:102A10002268830F00EA0A001065CBF800302046D8
:102A2000039900F005FB30050CD4E843000509D4F8
:102A3000236800204FF400621A65CBF8000020469E
:102A400000F000FBB00512D4E84380050FD42068E5
:102A500000234FF40078D0F8D820D0F8E010C0F868
:102A60005080CBF800301140204600F0E9FA3003E6
:102A70000CD4E843000309D4236800204FF400225B
:102A80001A65CBF80000204600F0D0FAF0030CD411
:102A9000E843C00309D4236800204FF480321A654C
:102AA000CBF80000204600F0C9FA70030CD4E843CC
:102AB000400309D4226800204FF480231365CBF82B
:102AC0000000204600F0B9FAB0030FD4E8438003B9
:102AD0000CD4236800204FF400321A65CBF80000B4
:102AE000D4F89C0040F08000C4F89C00B9F1000FBD
:102AF0000BD022684FEA997309EA0A001065CBF8F7
:102B0000003049462046FFF7F7FE5FB12268BB0F51
:102B100007EA0A001065CBF80030D4F89C0038436F
:102B2000C4F89C003C492068884268D160688146AE
:102B30008068800763D0D9F82060D9F82410D9F8CC
:102B40002080D9F82400D9F820C0D9F82470D9F809
:102B50002030D9F82450D9F8202003F4FC4306F0A3
:102B60000F0AD9F824601D40D9F824B008F03008C5
:102B70000CF4C07C02F4F02211EA0A0100EA080811
:102B800007EA0C0706EA0206D9F820A004D0C9F823
:102B90002010204600F04EFAB8F1000005D0616820
:102BA00008624146204600F047FA6FEA0B004006F3
:102BB0000ED46FEA0A0040060AD460684021C36B55
:102BC000C26B01622046190C02F03F0200F033FA9A
:102BD0002FB1606807623946204600F02AFA35B105
:102BE00060680562D4F89C002843C4F89C0036B1A4
:102BF00060680662D4F89C003043C4F89C00D4F8A6
:102C00009C00002802D02046FFF775FEBDE8FF9F1C
:102C100010A80040FFFFCF3F00A000402DE9F04189
:102C200094B08D494C2204466846FDF70DFD64B111
:102C30008A4D2068A84202D100F58070606094F847
:102C400098004FF0000820B108E0012014B0BDE862
:102C5000F081204684F8998000F002F920688169AB
:102C600021F01001816100F003FB0327064604E018
:102C700000F0FEFA801B0A2811D82068806900073E
:102C8000F6D42068816941F00101816100F0F0FA19
:102C900006460DE000F0ECFA801B0A2808D9D4F8AB
:102CA0009C0040F00100C4F89C0084F89870CCE7C8
:102CB00020688069C007EDD02068816941F0020179
:102CC0008161207C01282068816937D041F0400172
:102CD0008161607C01282068816932D021F48041C3
:102CE0008161A07C0128206881692DD041F4805148
:102CF00081612068A268816921F44071114381617A
:102D00002068816921F0A40181612068016921F0B6
:102D100010010161E068012819D010B302281BD00E
:102D20002068816941F0800181612068016941F07A
:102D300010010161E06803280ED012E021F040018B
:102D4000C6E741F48041CBE721F48051D0E7206809
:102D5000816941F0040103E02068816941F02001AC
:102D60008161207E6FF0FF02D4E90773A68A110209
:102D7000400602EB0727A0F10070384327685B1E6E
:102D8000184301EB06463043F861A068B0F5407F78
:102D900011D104F12800A68C6FF00F0C89C801EB4B
:102DA0000641401E02EB0322104322680CEB07137E
:102DB00018430843D060206E30B12068626ED0F8AE
:102DC000C0101143C0F8C010D4E917126846D142B0
:102DD00009D02168A36E51F8C82F50F8233022F093
:102DE00007021A430A60216C49B12168626C51F8EC
:102DF000BC3F50F8226023F0070232430A60A16C06
:102E000051B12168E36C51F8BC2F50F8233022F007
:102E1000700242EA03120A60216D51B12168626DAD
:102E200051F8BC3F50F8220023F4E06242EA00204F
:102E300008602068A84204D16068816821F003011D
:102E40008160C4F894800121C4F89C8084F89810B3
:102E50002046FDF799FEF9E604C1000800A00040F5
:102E60002DE9F047B4B0814614212EA8FDF726FCC9
:102E7000B8216846FDF722FC664C0026D9F8000010
:102E80004FF08051644A0C3C614F4FF00208614D95
:102E90009042DFF888A14FF0090938D100201B913A
:102EA0004A13CDE90020684601F0A4FE08B1FDF701
:102EB00036FE3868401C3860012807D1286840F485
:102EC00080702860286800F480703390206840F09B
:102ED00008002060206803222E922EA900F008002E
:102EE000CDE92F863196CDE93290504600F0ACF80E
:102EF00000220521132000F059FA132000F048FAAF
:102F000000220521152000F051FA15203BE0444A2B
:102F100090423DD100201B914FF40042CDE90020AA
:102F2000684601F067FE08B1FDF7F9FD3868401CFE
:102F30003860012807D1286840F48070286028682C
:102F400000F480703390206840F002002060206818
:102F500060222E922EA900F00200CDE92F86319634
:102F6000CDE932902F4800F06FF80022052114209F
:102F700000F01CFA142000F00BFA002205211620A4
:102F800000F014FA162000F003FA34B0BDE8F08720
:102F9000254A9042F9D100201B914FF40042CDE91F
:102FA0000020684601F026FE08B1FDF7B8FD38683C
:102FB000401C3860012807D1286840F480702860E0
:102FC000286800F480703390206840F0080020608A
:102FD00020684FF440512E91052200F00800CDE901
:102FE0002F862EA93196CDE93220504600F02CF8DC
:102FF000002205219F2000F0D9F99F2000F0C8F998
:1030000000220521A02000F0D1F9A020BBE700009C
:1030100000000024EC44025800A00040000C0258BC
:1030200000A400400004025800D4004070477047DC
:1030300070477047704770477047704770477047D8
:1030400070477047704700002DE9F84F03247A4D10
:1030500000234FF001094FF0B04B4FF00F0AE4E0AE
:1030600009FA03F6324078D00F7907F00307012FF1
:1030700001D0022F1AD187684FEA430ED1F80CC055
:1030800004FA0EF827EA08070CFA0EFC4CEA070CC3
:10309000C0F808C0476891F804C0B743CCF3001CDF
:1030A0000CFA03FC4CEA070CC0F804C00E79F64396
:1030B000B6070BD0C6684FEA43088F6804FA08FCCD
:1030C00026EA0C0607FA08F73743C7600E7906F0C0
:1030D0000306022E12D1DE080F694FEA437C00EB93
:1030E0008606B646366A4FEADC6C0AFA0CF807FA2E
:1030F0000CF726EA08063743CEF820700F790668E9
:103100004FEA430807F0030704FA08FC07FA08F738
:1031100026EA0C06374307604E6816F4403F1CD081
:10312000464E376847F00207376036689F0706F05B
:103130000206009623F0030606F1B046B6463F0F9E
:10314000D6F80864DFF8F8800AFA07FC404526EA5A
:103150000C0603D14FF0000C3AE065E0DFF8E4C064
:10316000604502D14FF0010C32E0DFF8DCC0604571
:1031700002D14FF0020C2BE0DFF8D0C0604502D145
:103180004FF0030C24E0DFF8C8C0604502D14FF0D7
:10319000040C1DE0DFF8BCC0604502D14FF0050C07
:1031A00016E0DFF8B4C0604502D14FF0060C0FE026
:1031B000DFF8A8C0604502D14FF0070C08E0DFF847
:1031C000A0C0604502D14FF0090C01E04FF00A0C9D
:1031D0000CFA07FC4CEA060CCEF808C44F68DBF882
:1031E0000060FF0226EA020600D516435F46CBF8D0
:1031F0000060D1F804C0DBF804605FEA8C2C26EA9A
:10320000020600D516437E606E684F6826EA020605
:10321000BF0300D516436E602E684F6826EA02068B
:10322000FF0300D516432E605B1C0A6832FA03F6D2
:103230007FF416AFBDE8F88F80000058F4440258C0
:10324000000002580004025800080258000C0258FE
:10325000001002580014025800180258001C0258AE
:10326000002402580AB1816170470904FBE700009D
:1032700001488068704700003800002402488168D7
:10328000027811448160704738000024032010B593
:1032900000F0ACF802F0EEFA0F4A10491468136817
:1032A000C4F3032203F00F038A5CC95C02F01F021F
:1032B00001F01F01D0400A4A20FA01F111600949CA
:1032C00008600F2000F010F808B1012010BD00F0D8
:1032D0004DF8002010BD00001844025878C10008C5
:1032E000480000244400002410B5102804468AB089
:1032F0002AD200220146A12000F058F8A12000F0B7
:1033000047F8154804601548016841F08071016074
:10331000006808A900F080700990684602F036FA4B
:1033200002F096FA0E49400000220E4CB0FBF1F17B
:103330000D4840F2E7330460C0E90332491EC0E99A
:10334000011203F0B1F810B101200AB010BD064817
:1033500003F0DCF8F9E700003C000024EC440258DC
:1033600040420F0000E000409C070020074882B068
:10337000016841F002010160006800220F2100F0A5
:1033800002000090901E02B000F010B8F444025801
:10339000002809DB410900F01F028900012001F12A
:1033A000E0219040C1F80001704700000E4BF0B4DE
:1033B0001B680D46C3F30223C3F10706042E00D990
:1033C0000426191D072901D2002300E0DB1E012479
:1033D00004FA06F19C40491E2940641E994014409D
:1033E0002143F0BC07F031BA0CED00E0064900F0D3
:1033F000070210B54FF6FF040868044B204040EA6E
:1034000002201843086010BD0CED00E00000FA0532
:103410002DE9F04F02688346FF484FF0000A8DB057
:103420000C468242564602D10025012001E00125CA
:103430000020E8460027814607EB47017F1C08EB88
:10344000C101F8B204F0BCFB20B108204FF0010A22
:10345000CBF85400FFB2022FEED3BAF1000F7CD1AB
:10346000DFF8B4E3DEF80000C00707D0DEF8001094
:1034700046F0010621F00101CEF80010E74800688F
:10348000C00706D0E54846F00206016821F00101B8
:10349000016005EB45030C93E148424608EBC3038A
:1034A000DFF880B30121DC469F6800EB8707D7F87F
:1034B000008428F48078C7F80084DBF80070FF07E8
:1034C00032D0DCF80070B9F1010F27F00107CCF819
:1034D00000705CD1069B00EB8303D3F8007447F0C7
:1034E0000207C3F80074079B3BB100EB8303D3F8DA
:1034F000007447F02007C3F80074099B4BB121EA20
:10350000030700EB8703D3F8047447F48027C3F85C
:1035100004740A9BDBB321EA030700EB8703D3F8AB
:10352000047447F0806730E00C9F52F8377077B32F
:1035300000EB8707D7F800C42CF0010CC7F800C4D3
:103540005F683FB100EB8707D7F800C42CF0100C80
:10355000C7F800C4D3F80CC000E05AE1BCF1000F7A
:1035600009D021EA0C0700EB8707D7F804C42CF434
:10357000803CC7F804C41B694BB121EA030700EB88
:103580008703D3F8047427F08077C3F8047409EB39
:103590004903D4F800C0CDF830C0914652F83370DA
:1035A000BC451BD009EBC302D4F808C0D2F8088090
:1035B000C44513D0D4F804C0D2F80480C44502D165
:1035C000BCF1000F0AD1D4F80CC0D2F80C80C4456D
:1035D00004D0D4F810C01269944551D10C9ABA4263
:1035E00019D109EBC302D4F804C0D2F80480C44551
:1035F00011D1D4F80CC0D2F80C80C4450BD1D4F84A
:1036000010C01269944506D1DBF8003043F0010385
:10361000CBF8003034E000EB870709EBC302D7F8A2
:10362000003423F00103C7F8003453683BB100EBCA
:103630008303D3F8007427F01007C3F8007493686D
:1036400000EB8303D3F8007427F48077C3F8007489
:10365000D3684BB121EA030700EB8703D3F8047466
:1036600027F48037C3F8047412694AB121EA0203CF
:1036700000EB8302D2F8043423F08073C2F80434E0
:10368000A3685A4600EB8303D3F8007427F440770D
:1036900047EA452747F48077C3F80074DBF800C099
:1036A00063695F1ECCF3074C674508D95E4FD2F8BB
:1036B00000C007EB03472CF47F033B431360126801
:1036C000D207226800EB8202D2F800343FD023F008
:1036D00003035B1CC2F8003462684AB100EB82024B
:1036E000D2F8003423F0300343F01003C2F8003462
:1036F000E268D3030AD521EA020300EB8302D2F881
:10370000043423F4E02343F480330AE05AB121EA7D
:10371000020300EB8302D2F8043423F0E06343F0A9
:103720008073C2F804342269D30307D5914300EBB8
:103730008100D0F8041421F4E0214AE0F2B391436F
:1037400000EB8100D0F8041421F0E0614EE001EBC1
:10375000450723F003033B43C2F8003462685AB1C3
:1037600000EB8202D2F8003423F0300343EA451321
:1037700043F01003C2F80034E268D3030CD521EA09
:10378000020300EB8302D2F8043423F4E02343EA7B
:10379000854343F480330CE06AB121EA020300EB75
:1037A0008302D2F8043423F0E06343EA856343F0F4
:1037B0008073C2F804342269D30300E01AE00BD509
:1037C000914300EB8100D0F8041421F4E02141EA98
:1037D000854141F440310BE062B1914300EB81003F
:1037E000D0F8041421F0E06141EA856141F04071B4
:1037F000C0F80414F00705D0DEF8001041F0010114
:10380000CEF80010B00704D50448016841F001016A
:1038100001600DB0504609E00050005200A0005277
:1038200000B0005200B400520000FFFFBDE8F08F6E
:10383000F8B500250446FFF71BFD064624B100201D
:103840006065206D10B170E001256EE0204600F04B
:1038500073F841F28830A065258A6FF0FF01226875
:10386000D4F814C00F02636B07EB0545E06801EB69
:103870000C27D4F81CC0184393683D432D4F2843B0
:103880003B4040EA0C00184390602068236AC268FD
:1038900022F4E0221A43C2602368228EA06B40EA21
:1038A000024018612268E06B5061D4E900030268AD
:1038B00001EB032322F4F85119430160A06D0022AB
:1038C000202133460090204604F0E8F905002CD171
:1038D0002068626AC168521E21F0FF011143C16075
:1038E0002068A268016821F040011143016020684E
:1038F000D4E90A12D0F80831114323F0A042114351
:10390000C0F808112068016841F001010160A06958
:10391000022804D12068816841F002018160E068DA
:10392000B0F1806F03D0022020652846F8BD012049
:10393000FAE70000F4F8E0F82DE9F043B5B00446EA
:1039400014216846FCF7BAFEB82106A8FCF7B6FEBB
:103950004749206888427DD1002019904FF00071BE
:103960000446CDE9061006A801F044F908B1FDF7B8
:10397000D6F84048016841F400110160016801F483
:1039800000110591016841F400210160006800F414
:103990000020059037480C30016841F001010160BA
:1039A000016801F001010591016841F00201016027
:1039B000016801F002010591016841F01001016008
:1039C000016801F010010591016841F008010160F2
:1039D000006802250927009500F00800DFF89880AC
:1039E000032603966946CDE90470CDE901544046AB
:1039F000FFF72AFB062102940820CDE90361CDE9F7
:103A0000000569464046FFF71FFB0121DFF86C9077
:103A100002AA4FF00408CDE900156946484682E83D
:103A20005001FFF711FB02AA6946484682E8D00020
:103A3000CDE90085FFF708FB0B2111484FF4006822
:103A4000CDF80080CDE90361CDE901546946FFF767
:103A5000FBFA00E008E002AA0A48694682E8D000C2
:103A6000CDE90085FFF7F0FA35B0BDE8F08300003E
:103A700000A00052D444025800000258000402582A
:103A800000100258000C025801680123C0F8D83415
:103A9000002280F8CC248869044A40F000608861E4
:103AA000486D104348650020704700000300001077
:103AB00070470068416200207047F0B503685D6A96
:103AC00039B19F6A4C1E00204FF4827605EB1745F2
:103AD0000BE045EA0240986210E0471C06EB8000CC
:103AE00053F800C0F8B205EB1C45A042F5D34FF4E3
:103AF000807000EB810045EA02421A500020F0BDC0
:103B0000D0F8E00405F0EDBD01EBC10200EB82024C
:103B1000D0F8E004126A05F040BD01EBC10200EBF1
:103B20008202D0F8E004D2F8602205F092BDD0F80D
:103B3000E00405F0D8BD0A0601F00F0101EBC10158
:103B400000EB810101D5143101E001F51571006828
:103B500006F0C6BC01F00F020B0670B502EBC20105
:103B600004464FF001004FF0000504EB810102D53F
:103B70004875143103E081F8555201F515710A704A
:103B800094F89424012A08D084F89404206806F05C
:103B9000C5F9002084F8945470BD022070BD70B542
:103BA0000279044601F00F00904201D9012070BD56
:103BB00001F00F024FF000050B0602EBC2014FF0BF
:103BC000010204EB810102D54A75143103E081F84A
:103BD000555201F515718D70087094F89404012800
:103BE00008D084F89424206806F002FB002084F8B2
:103BF000945470BD022070BD01F00F0101EBC101B2
:103C000000EB8100D0F8680270472DE9F04101F027
:103C10000F0604460D064FF0010006EBC6014FF0FB
:103C2000000504EB810102D54875143103E081F8E9
:103C3000555201F51571C2F30A024F780B718A6073
:103C40000E7007B14E83022B00D14D7194F894246D
:103C5000012A09D084F89404206806F0A7F82846C1
:103C600084F89454BDE8F0810220FBE770B501F0C0
:103C70000F05002405EBC50100EB810101F518716A
:103C800081E81C0001F80B4C01F80C5D8379012BD5
:103C900000D1CA618279006806F002FB002070BD85
:103CA00070B50D460179044605F00F00884201D930
:103CB000012070BD29064FF000064FF0010206D525
:103CC00000EBC00104EB81014A75143107E005EBFC
:103CD000C50104EB810181F8556201F515718A7007
:103CE000087094F89404012807D084F8942420687C
:103CF00006F0AAFA280702D007E0022070BDA179D9
:103D000004F29C42206806F047FA002084F894648C
:103D100070BD70B501F00F04002504EBC40101264D
:103D200000EB8101203181E82C0001F80B6C01F8D7
:103D30000C4D8379012B00D1CA618279006806F0AD
:103D4000AFFA002070BD00002DE9FC5F0568044655
:103D5000284606F061FC00287ED1206806F088FC29
:103D6000002879D0D5F80808C0F30D20C4F8D40491
:103D7000206806F07DFC800704D52068416901F0C9
:103D800002014161206806F073FCC10604F29C4008
:103D9000009035D52068816921F0100181612F6A7A
:103DA00007F00F01C7F3434001EBC101022804EB08
:103DB000810606F5157602D0062812D01BE047F6DC
:103DC000F070074217D0C7F30A12F1681746284669
:103DD00006F052FC7169F068394471613844F06052
:103DE00009E000990822284606F046FC7069C7F3EE
:103DF0000A11084470612068816941F010018161F5
:103E0000206806F035FC00034FF0080B4FF0000A65
:103E10004FF001097CD52068002606F008FC074613
:103E200074E0F80770D02068F1B206F019FC804603
:103E3000C00707D005EB4611C1F8089B3146204664
:103E400003F056FF5FEA087024D505EB4611C1F870
:103E500008BBFA49206800E03EE2026C00EB461025
:103E600001928A42D0F8081B05D9090403D54FF402
:103E70000041C0F8081B204600F001FBEF49019803
:103E8000884207D9A079012804D120680121009A2D
:103E900006F082F95FEAC86004D505EB46111020F0
:103EA000C1F8080B5FEA88701DD56869000605D562
:103EB000D5F8040840F48061C5F8041806EBC60084
:103EC00004EB800090F8571200F51570012905D118
:103ED00080F803A02046F1B200F004FA05EB461189
:103EE0000220C1F8080B5FEA886004D505EB461193
:103EF0002020C1F8080B5FEA884005D505EB461184
:103F00004FF40050C1F8080B7F08761C002F88D1B1
:103F1000206806F0ADFB40036ED5206806F080FBFC
:103F20000026074666E0F80762D02068F1B206F086
:103F300085FB8046C00723D0D5F8342806F00F0C47
:103F400005EB461309FA0CF08243C5F83428C3F890
:103F50000899A07901280FD106EBC60004EB800078
:103F6000D0E907211144016236B9606A20B920689E
:103F70000121009A06F010F92046F1B2FFF7C4FDC6
:103F80005FEA087003D505EB4611C1F808B95FEA8E
:103F9000C86004D505EB46111020C1F808095FEA96
:103FA000486004D505EB46114020C1F808095FEAD6
:103FB000887016D53146284606F003FB06EBC6008E
:103FC00004EB8000C17D1430012905D180F803A0E5
:103FD0002046F1B200F082F905EB46110220C1F84B
:103FE00008095FEA086003D53146204603F0E6FE83
:103FF0007F08761C002F96D1206806F039FB002838
:1040000011DAD5F8040820F00101C5F8041894F875
:10401000CC0401283BD0204600F016FA2068416904
:1040200001F000414161206806F022FB00050BD53C
:10403000D5F80808C00702D0204600F049FA2068E9
:10404000416901F400614161206806F011FB000143
:104050000AD52068416901F00061416194F8CC04FF
:10406000E0B1204600F034FA206806F001FBC004FD
:1040700072D5D5F8040820F00100C5F804082068BE
:10408000102106F09EFA00214FF67F322DE000212C
:10409000204684F8CCA4FFF70BFDBFE784F8CC944E
:1040A0002068406D0121C0F38300C4F8D00420468D
:1040B000FFF7FEFCD8E700BF05EB4110C0F8082968
:1040C000D0F8003923F40013C0F80039C0F8082BE9
:1040D000D0F8003B23F40013C0F8003BD0F8003BBD
:1040E00043F00063C0F8003B491C20798842E3D8C4
:1040F000D5F81C0840F00111C5F81C18E07B68B128
:10410000D5F8840840F00B01C5F88418D5F84408A8
:1041100040F00B012846C5F844180DE0D5F8140806
:1041200042F22B010843C5F81408D5F8100840F0F6
:104130000B012846C5F81018D0F8000820F4FE61DD
:10414000C5F80018A1792068009A06F025F82068C3
:10415000416901F480514161206806F089FA8004C8
:1041600016D5206805F062FE206806F048FAE07176
:1041700001F03AFB23680146E279184606F0DCFAC2
:10418000204600F04BF92068416901F4005141617B
:10419000206806F06DFA000707D5204600F058F9B0
:1041A0002068416901F008014161206806F060FA69
:1041B000000615D5A869012620F08001A9610CE050
:1041C00006EBC60004EB800090F85702012803D1EB
:1041D0002046F1B2FFF7AFFC761C2079B042EFD851
:1041E000206806F045FAC0021FD501264F4614E0AC
:1041F00006EBC60005EB461304EB8001D3F800097B
:104200000A7E012A08D1002806DAF0B2CF7540F004
:1042100080012046FFF78FFC761C2079B042E7D85A
:104220002068416901F480114161206806F020FA9C
:10423000800234D501204A4629E000000A30544F5C
:1042400000EBC00305EB401604EB8301D6F8006BCE
:1042500091F85832012B19D1002E17DA94F8D43482
:10426000C6F3004603F00103B3420FD181F8572291
:10427000A96941F08003AB616969090606D4D5F8E4
:10428000040840F40070C5F8040803E0401C2179DC
:104290008142D5D82068416901F40011416120684C
:1042A00006F0E6F9400007D52046FFF729FC206814
:1042B000416901F080414161206806F0D9F9400769
:1042C0000AD520684568680702D52046FFF72FFC0D
:1042D0002068416829434160BDE8FC9FD0F8E004B4
:1042E00005F059BAD0F8E00405F069BAF8B5040051
:1042F00004D094F89504002510B106E00120F8BD23
:10430000204684F8945400F057F8032084F895046C
:10431000206805F03BFF207C8DF8000094E80F003A
:1043200005F092FD0226B0BB2068002106F0C4F91A
:1043300088BB002001270CE000EBC001421C04EB0D
:1043400081014F750D76CD610D624D620875C8858E
:10435000D0B221798142EFD8002011E000EBC001FA
:10436000421C04EB810181F8555281F85852C1F882
:104370005C52C1F86052C1F8645281F85402D0B264
:1043800021798142EAD8207C8DF8000094E80F0062
:1043900005F046FE10B184F89564AFE7207B6574A4
:1043A00084F89574012802D12046FFF76DFB206840
:1043B00005F028FE0020F8BD10B5B0B00446B821C5
:1043C0006846FCF77BF913492068884220D1002019
:1043D0004FF480214FF440122192CDE9001068463D
:1043E00000F008FC08B1FCF79AFB00F0B3F80A48AB
:1043F000016841F00071016000680022052100F0B1
:1044000000702E904D20FEF7D1FF4D20FEF7C0FF2B
:1044100030B010BD00000440D844025870B50446C6
:10442000C079012570B1022801D0FCF778FBD4F8DF
:10443000E004294605F032FAD4F8E004BDE8704003
:1044400005F0E6B90025F2E7D0F8E00405F00FBA70
:10445000D0F8E00405F015BA10B5044690F89404BD
:1044600001280AD00120617484F89404206806F0C1
:1044700052F9002084F8940410BD022010BDD0F839
:10448000E02400F29C41104605F014BA10B590F8F3
:10449000941404460068012909D0012184F8941479
:1044A000C168490609D5617B012902D005E00220D7
:1044B00010BD816B41F480318163206806F05FF8A4
:1044C000206805F091FD002084F8940410BD0000E0
:1044D00010B50446D0F8E00405F02EFA2068D0F8B4
:1044E000001E41F00101C0F8001EE07A002804D04F
:1044F0000248016841F00601016010BD10ED00E0C6
:10450000134970B50A68D243520705D5096801F00E
:104510000701814213D118E00A6822F00702024322
:104520000A60FEF7A5FE0A4D4FF47A760446083D70
:1045300007E000BFFEF79CFE001BB04201D901203E
:1045400070BD2868C0438004F4D4002070BD000012
:104550000C4802580248016841F0807101607047C0
:104560000C48025810B501F03FF905490968054AA1
:10457000C1F30211515C01F01F01C84010BD0000E1
:104580002044025878C100084A4930B5494C0B1DF7
:104590000A680C3409681D68246802F0030305F0FA
:1045A0000102C1F30511C4F3CC04002914FB02F28B
:1045B00000EE102AF8EE400A76D0414A9FED3E1AEE
:1045C000DFED3E1AB7EE000A23B1012B5AD0022BC1
:1045D00018D15CE0374C283C23689B0612D5394B38
:1045E000246801EE901A1168C4F3C104F8EE612A40
:1045F000E34001EE903AC1F30801F8EE611A81EE52
:10460000A22A07E002EE101A1168F8EE422A81EEA3
:10461000A22A45E001EE901A1168F8EE611A40EE08
:10462000811A71EE800A62EE200AC1F3462101EE82
:10463000101AB8EE411A31EE001AC0EE811ABCEE23
:10464000E11A80ED001A1168C1F3064101EE101A5B
:10465000B8EE411A31EE001AC0EE811ABCEEE11A32
:1046600080ED011A1168C1F3066101EE101AB8EE6F
:10467000411A31EE000A80EE801ABCEEC10A80EDCC
:10468000020A30BD01EE901ADFED0F2A03E001EEC1
:10469000901ADFED0E2A1168F8EE611A82EEA12A57
:1046A000C1F30801B6E7FFE70021016041608160C6
:1046B00030BD000028440258000000390024744C2A
:1046C000304402580090D0030024744A001BB74BBA
:1046D000494930B5484C0B1D0A68143409681D68F7
:1046E000246802F00303C5F30012C1F30531C4F3DB
:1046F000CC04002914FB02F200EE102AF8EE400A66
:1047000075D03F4A9FED3D1AB7EE000A6BB1DFED61
:104710003D1A012B01D0022B64D002EE101A116851
:10472000F8EE422A81EEA22A21E0334C283C23688D
:104730009B0612D5344B246801EE901A1168C4F31D
:10474000C104F8EE612AE34001EE903AC1F308019A
:10475000F8EE611A81EEA22A0BE001EE901ADFED6D
:104760002B2A00BFF8EE611A116882EEA12AC1F36C
:10477000080101EE901A1168F8EE611A40EE811AF4
:1047800071EE800A62EE200AC1F3462101EE101A92
:10479000B8EE411A31EE001AC0EE811ABCEEE11AF1
:1047A00080ED001A1168C1F3064101EE101AB8EE4F
:1047B000411A31EE001AC0EE811ABCEEE11A80ED0A
:1047C000011A1168C1F3066101EE101AB8EE411A20
:1047D00031EE000A80EE801ABCEEC10A80ED020ABA
:1047E00030BD04E001EE901ADFED092ABAE700219E
:1047F000016041608160F3E72844025800000039FD
:10480000384402580024744A0090D0030024744CA9
:10481000001BB74B494930B5484C0B1D0A681C3486
:1048200009681D68246802F00303C5F30022C1F380
:104830000551C4F3CC04002914FB02F200EE102A47
:10484000F8EE400A75D03F4A9FED3D1AB7EE000AD8
:104850006BB1DFED3D1A012B01D0022B64D002EECB
:10486000101A1168F8EE422A81EEA22A21E0334C98
:10487000283C23689B0612D5344B246801EE901A1D
:104880001168C4F3C104F8EE612AE34001EE903AE6
:10489000C1F30801F8EE611A81EEA22A0BE001EEE5
:1048A000901ADFED2B2A00BFF8EE611A116882EE34
:1048B000A12AC1F3080101EE901A1168F8EE611AFD
:1048C00040EE811A71EE800A62EE200AC1F34621A1
:1048D00001EE101AB8EE411A31EE001AC0EE811A3C
:1048E000BCEEE11A80ED001A1168C1F3064101EE39
:1048F000101AB8EE411A31EE001AC0EE811ABCEE61
:10490000E11A80ED011A1168C1F3066101EE101A77
:10491000B8EE411A31EE000A80EE801ABCEEC10AF0
:1049200080ED020A30BD04E001EE901ADFED092AA5
:10493000BAE70021016041608160F3E72844025832
:1049400000000039404402580024744A0090D0030B
:104950000024744C001BB74B2DE9F04FA14A0546CB
:10496000DFF87CA280F48070DFF8809289B01311A8
:104970009F4C08439C48AAF104064FF0805C4FF01E
:10498000005828D0DFF858B285F480670F430BF148
:10499000080B4FD085F400670F4360D085F4805733
:1049A0000F4372D085F400570F434FF480394FF412
:1049B000003E69D085F400270F4373D085F480371B
:1049C0000F4370D085F480460E436DD085F40042CD
:1049D0000A436AD02AE0DAF8001001F0070105293D
:1049E00024D2DFE801F0F9AA6A259F0006A8FFF7A4
:1049F000CBFD079809B0BDE8F08F6846FFF768FE69
:104A00000098F7E703A8FFF705FF0398F2E720688F
:104A1000C0F3C10022FA00F0ECE72268D2056ED59F
:104A200061456CD11846E5E74145E3D00020E1E758
:104A30004846DFE7DBF8001001F46001B1F5800FB4
:104A40003BD005DC00294AD0B1F5001FEED174E05F
:104A5000B1F5C00FECD0B1F5000FE7D162E0DBF8A3
:104A6000001001F0E061B1F1007F26D004DCB1B3A9
:104A7000B1F1807FDAD160E0B1F1407FD8D0B1F1FF
:104A8000806FD3D14EE000E01BE0DAF8001001F4B3
:104A9000E041B1F5005F10D008DC01B3B1F5805FF3
:104AA000C4D14AE035E058E065E088E0B1F5405F08
:104AB000BED0B1F5804FB9D134E020688000B5D5C3
:104AC000A0E7DAF8001001F4E021B1F5403F6DD025
:104AD00006DC61B149457BD07145A7D158E07BE048
:104AE000B1F5802F66D0B1F5A02F9FD10DE000F079
:104AF0009DFE7FE76846FFF7EBFD01987AE728E027
:104B000003A8FFF787FE049874E7216889038AD415
:104B10008CE7DBF8001011F440310ED0494510D07D
:104B2000714583D13168256801F040516D077FF5EB
:104B300074AF00297FF471AF69E720680001E7D501
:104B40005BE720688000E3D503A8FFF763FE0598C4
:104B500050E722689203DBD566E7306810F48030B6
:104B60003AD04845D4D120680001D1D56846FFF736
:104B7000AFFD02983EE7DBF8001001F0E041B1F133
:104B8000405F13D008DC71B1614521D04145BFD1F0
:104B900020688000B4D449E7B1F1804F0AD0B1F168
:104BA000A04FB2D042E7FFF7DDFC23E720684007C3
:104BB000AED52CE72068C005AAD533E708E0DAF8BF
:104BC000001011F04051A0D0614505D041459FD162
:104BD000206800018ED429E72068800198D505E778
:104BE000504402580090D00300366E010080BB0094
:104BF000004402582DE9FE4F0546DFF800A450F8A6
:104C0000081B0024FD4FC943019005F128002646EA
:104C10000AF1240A009008011DD4686E50B1B0F565
:104C2000801F0CD0B0F5001F0ED0B0F5401F1ED075
:104C300001240FE0386840F40030386017E0019834
:104C4000022103F00DF903E00098022103F098F926
:104C500004000CD026462888C043C00523D4A86D84
:104C600005281ED2DFE800F00C11161B1B006A6E2F
:104C7000DAF8001021F440111143CAF80010EAE7F5
:104C8000386840F40030386009E00198002103F0F2
:104C9000E7F803E00098002103F072F90446C4B17C
:104CA00000E0012426462888DFF85083C04308F13D
:104CB0002C0840052FD4D5F8A400B0F5C00F28D09B
:104CC00010DCB8B1B0F5001F19D0B0F5800F0FD1CE
:104CD0001AE0AA6DDAF8001021F007011143CAF8B2
:104CE0000010E0E7B0F5000F13D0B0F5200F10D0A2
:104CF00001240FE0386840F40030386009E0019882
:104D0000002103F0ADF803E00098002103F038F92A
:104D1000044694B126462888C043000530D4D5F80F
:104D2000A800B0F1407F29D011DCC0B1B0F1807F84
:104D30001AD0B0F1007F10D11BE0D5F8A420D8F82C
:104D4000001021F460011143C8F80010E3E7B0F14E
:104D5000806F13D0B0F1A06F10D001240FE038683D
:104D600040F40030386009E00198002103F078F841
:104D700003E00098002103F003F9044694B12646AD
:104D80002868DFF878B2C0430BF1200B80011FD4F4
:104D9000E86CD8B110280FD0202812D0302815D0B8
:104DA000012414E0D5F8A820D8F8001021F0E06123
:104DB0001143C8F80010E3E7386840F40030386069
:104DC00004E00198022103F04BF8044674B1264632
:104DD0002888C043C0042BD4E86DB0F5005F20D014
:104DE0000DDCA0B1B0F5805F0FD115E0EA6CDBF807
:104DF000001021F030011143CBF80010E8E7B0F5C6
:104E0000405F13D0B0F5804F10D001240FE0386818
:104E100040F40030386009E00198002103F020F8E8
:104E200003E00098002103F0ABF804468CB126465D
:104E30002888C043800429D4286EB0F5403F23D091
:104E400010DC08B3B0F5803F14D0B0F5003F0FD1AF
:104E500015E0EA6DDAF8001021F4E0411143CAF8D8
:104E60000010E5E7B0F5802F0ED0B0F5A02F0BD0E5
:104E700001240AE00198012102F0F2FF03E000980A
:104E8000012103F07DF8044694B126462888C043EA
:104E900040042AD4D5F8AC00B0F1405F23D010DC38
:104EA00008B3B0F1805F14D0B0F1005F0FD115E00E
:104EB0002A6EDAF8001021F4E0211143CAF800103C
:104EC000E4E7B0F1804F0ED0B0F1A04F0BD0012439
:104ED0000AE00198012102F0C3FF03E000980121DC
:104EE00003F04EF8044674B126462888C0430004F7
:104EF0001FD4E86ED8B1B0F1805F0ED0B0F1005F82
:104F000010D0012414E0D5F8AC20D8F8001021F01E
:104F1000E0411143C8F80010E7E7386840F400307A
:104F2000386004E00198012102F09AFF044674B150
:104F300026462868C043C0011ED4A86CD0B1012801
:104F40000ED0022811D0032814D0012413E0EA6EF9
:104F5000DAF8001021F040511143CAF80010E8E7D8
:104F6000386840F40030386004E00198022102F013
:104F700077FF04466CB126462868C043400255D4EA
:104F80001F48016841F480710160FEF771F98146A4
:104F90000EE0AA6CDBF8001021F003011143CBF8FE
:104FA0000010E9E7FEF764F9A0EB090064283BD89C
:104FB00013480068C005F5D5BCBBDFF84090B5F8D4
:104FC000B01009F14409D9F8000001F4407100F46F
:104FD0004070884211D0D9F80010D9F8002021F48F
:104FE000407142F48032C9F80020D9F8002022F440
:104FF0008032C9F80020C9F8001003E02C440258A0
:1050000000480258D5F8B000B0F5807F19D1FEF7FE
:105010002FF9029011E000BFFEF72AF90299411A18
:1050200041F28830814208D9032426462878DFF8E7
:105030001494C043C00721D03CE0D9F80000800799
:10504000EAD5D5F8B010C1F301200328FE480DD0F1
:10505000016821F47C510160B5F8B020D9F8001046
:10506000C2F30B021143C9F80010DFE7F74A0368E7
:1050700002EA111223F47C511143ECE7A86F1828BF
:1050800016D005DCA0B1082808D0102804D10AE009
:1050900020280DD028280BD001240AE001980121F6
:1050A00002F0DEFE03E00098012102F069FF0446F1
:1050B00064B126462878C04380071ED4686F06284E
:1050C00019D2DFE800F0160C11161616AA6FD9F8DF
:1050D000001021F038011143C9F80010EAE70198E7
:1050E000012102F0BDFE03E00098012102F048FF1B
:1050F00004467CB100E0012426462878C0434007DE
:105100001FD4D5F89000062819D2DFE800F0160C5D
:10511000111616166A6FD9F8001021F00701114315
:10512000C9F80010E9E70198012102F099FE03E0B7
:105130000098012102F024FF0446A4B100E00124FC
:1051400026462878C04380062BD4D5F88C00B0F1D1
:10515000405F24D011DC10B3B0F1805F15D0B0F106
:10516000005F10D116E0D5F89020D8F8001021F09B
:1051700007011143C8F80010E3E7B0F1804F0ED0EB
:10518000B0F1A04F0BD001240AE00198002102F0F9
:1051900067FE03E00098022102F0F2FE044694B19B
:1051A00026462878C04340062BD4D5F89800B0F5A1
:1051B000406F24D011DC10B3B0F5806F15D0B0F57E
:1051C000006F10D116E0D5F88C20D9F8001021F02E
:1051D000E0411143C9F80010E3E7B0F5805F0ED05D
:1051E000B0F5A05F0BD001240AE00198002102F085
:1051F00037FE03E00098022102F0C2FE044694B19B
:1052000026462878C04300062BD4D5F89C00B0F57C
:10521000C04F24D011DC10B3B0F5005F15D0B0F54D
:10522000804F10D116E0D5F89820D8F8001021F45E
:10523000E0511143C8F80010E3E7B0F5004F0ED07D
:10524000B0F5204F0BD001240AE00198002102F0B4
:1052500007FE03E00098022102F092FE044654B1DA
:1052600026462878C04300071ED4D5F88000B0F544
:10527000805F0AD00FE0D5F89C20D8F8001021F408
:1052800060411143C8F80010EBE70098022102F0DA
:1052900077FE00B10126D5F88020D9F8001021F45E
:1052A00040511143C9F800102878C043C00613D4F8
:1052B000D5F89400B0F5807F05D10098022102F066
:1052C0005FFE00B10126D5F89420D8F8001021F433
:1052D00040711143C8F800102868C043000316D479
:1052E000D5F8A00038B1B0F5803F09D0B0F5003F47
:1052F0000BD001240AE00198002102F0B1FD03E087
:105300000098022102F03CFE04468CB12646286833
:10531000C043400322D4D5F88400B0F5801F11D0DB
:10532000B0F5001F13D0B0F5401F15D0012414E0D4
:10533000D5F8A020D8F8001021F440311143C8F866
:105340000010E4E7386840F40030386004E000986A
:10535000012102F015FE04465CB126462868C043D0
:10536000C0031CD4286D70B1B0F5803F10D001246B
:1053700014E0D5F88420D9F8001021F4401111432D
:10538000C9F80010EAE7386840F40030386004E0FB
:105390000198022102F064FD0446DCB1264628682B
:1053A000C043800005D40098022102F0E9FD00B15D
:1053B00001262868C04380031BD4E86FB8B1B0F55C
:1053C000807F10D0B0F5007F11D0B0F5407F0ED0B7
:1053D00001240DE02A6DDBF8001021F48031114327
:1053E000CBF80010DBE7386840F4003038607CB35D
:1053F00026462868C043C00207D42A6FDAF8001096
:1054000021F000411143CAF800102868C04380020F
:1054100007D4AA6EDAF8001021F080711143CAF89F
:1054200000102868C043400009D40748016821F4EF
:10543000004101600168D5F8B4201143016028687B
:10544000C04306E05444025810440258CFFFFF0006
:105450001DE007D46A6DDBF8001021F040511143C4
:10546000CBF800102868C043000208D4D5F8882083
:10547000D9F8001021F440011143C9F8001028792F
:105480000024C04300F00100204309D00EE0EA6F81
:10549000D9F8001021F440711143C9F80010A8E7B1
:1054A0000198002102F0DCFC00B106462879C043D7
:1054B00000F00200204305D10198012102F0D0FC48
:1054C00000B106462879C04300F00400204305D10E
:1054D0000198022102F0C4FC00B106462879C043BD
:1054E00000F00800204305D10098002102F048FD9B
:1054F00000B106462879C04300F01000204305D1D2
:105500000098012102F03CFD00B106462879C04315
:1055100000F02000044304D10098022102F030FD85
:1055200000B916B10120BDE8FE8F0020FBE70000A6
:105530002DE9F05F04000F467ED0DFF83882D8F8FE
:10554000000000F00F00B8420CD2D8F8001021F093
:105550000F013943C8F80010D8F8000000F00F0020
:10556000B84269D12078844D40070AD5206929685E
:1055700001F07001884204D9296821F070010143CB
:10558000296020787C4E361D00070AD56069316895
:1055900001F07001884204D9316821F070010143A3
:1055A00031602078C0060AD5A069316801F4E06155
:1055B000884204D9316821F4E061014331602078E8
:1055C000DFF8B4B180060BF1080B0CD5E169584641
:1055D000DBF8002002F07002914204D9026822F048
:1055E00070020A430260207880070AD5E0682968C3
:1055F00001F00F01884204D9296821F00F0101430D
:1056000029602078C0073ED05B49A2682868183915
:1056100020F47060104328606068022818D00328C6
:1056200019D00968012819D0490700294ADADFF89A
:1056300048A1AAF1080A00E044E0DAF8002022F0CC
:1056400007020243CAF80020FDF712FE814612E06D
:1056500009688903E9E709688901E6E7C905E4E71C
:10566000FDF706FEA0EB090141F28830814202D924
:105670000320BDE8F09F6168DAF8000000F0380010
:10568000B0EBC10FECD1207880070AD5E06829681B
:1056900001F00F01884204D2296821F00F01014373
:1056A0002960D8F80010404601F00F01B9420BD92B
:1056B000016821F00F0139430160006800F00F001C
:1056C000B84201D00120D4E7207840070AD52069EC
:1056D000296801F07001884204D2296821F0700124
:1056E00001432960207800070AD56069316801F01C
:1056F0007001884204D2316821F0700101433160A9
:105700002078C0060AD5A069316801F4E0618842BA
:1057100004D2316821F4E0610143316020788006D1
:105720000CD5E1695846DBF8002002F07002914286
:1057300004D2026822F070020A43026000F09AF874
:105740000E492A682B68C2F3032203F00F038A5C18
:10575000C95C02F01F0201F01F01D040084A20FA84
:1057600001F111600749086007480068BDE8F05F73
:10577000FDF7BABD002000521844025878C1000855
:1057800048000024440000243C00002470B5144C60
:105790003F220260124A24680832131D114D04F0A2
:1057A0000704446016681C1D06F47066866016685F
:1057B00006F00F06C660126802F0700202611A68F5
:1057C00002F0700242611A6802F4E06282612268AB
:1057D00002F07002C261286800F00F00086070BD1E
:1057E000104402580020005230B500F043F80B4A34
:1057F0000B490C4B15681468C5F3032204F00F0421
:105800008A5C095D02F01F0201F01F01D040064AC8
:1058100020FA01F119601060084630BD18440258A2
:1058200078C10008480000244400002400B5FFF7B8
:10583000DBFF05490968054AC1F30211515C01F01B
:105840001F01C84000BD00001C44025878C1000878
:1058500000B5FFF7C9FF05490968054AC1F30221F0
:10586000515C01F01F01C84000BD00001C440258FB
:1058700078C10008454970B545480968434B103B5D
:1058800011F0380208D00111082A03D0102A0BD0D9
:10589000182A0BD0084670BD19688906FBD519680F
:1058A000C1F3C101C84070BD3A4870BD3749374D9A
:1058B00018310C1D24350A68096826682D6802F025
:1058C000030406F00102C1F30511C5F3CC0515FB75
:1058D00002F200EE102AB8EE400AE9B32F4ADFEDDB
:1058E0002E0AB7EE001A6CB1DFED2D1A012C01D093
:1058F000022C43D002EE101A1068F8EE422A81EE14
:10590000A22A1EE01C68A40611D51B6801EE901A9D
:105910001168C3F3C103F8EE612AD84001EE900A82
:10592000C1F30800F8EE611A81EEA22A0BE001EE45
:10593000901ADFED1C2A00BFF8EE611A106882EEA3
:10594000A12AC0F3080001EE900AF8EE611A40EEB9
:10595000201A31EE810A00E015E022EE000A1068FC
:10596000C0F34620401C00EE900AF8EE600A80EE7C
:10597000201ABCEEC10A10EE100A70BD01EE901A9A
:10598000DFED092AD8E7002070BD0000104402585E
:105990000090D00300366E010000003930440258F8
:1059A0000024744A0024744C001BB74BF0B50D461C
:1059B0001F49204C002887B016464FF000004FF0DA
:1059C00002020F684FF0030319D047F004070F607D
:1059D000096801F00401059111020091CDE901204F
:1059E000CDE9033014486946FDF72EFB206845EAEF
:1059F000C61120F07E400843206007B0F0BD47F09C
:105A000001070F60096801F0010105914FF48071F1
:105A10000091CDE90120CDE9033008486946FDF742
:105A200013FB2068354320F0FE702843E4E70000B4
:105A3000E04402581044025800080258000002587E
:105A40002DE9F05F04007DD0FF4F2078FE4D183720
:105A5000DFF8F483103DC00748D0D8F8000039685B
:105A600000F03800102815D0182803D101F00300E9
:105A700002280FD06068B0F5803F12D010B1B0F5A9
:105A8000A02F18D0286820F480302860286820F4DF
:105A9000802009E02868800328D560680028D2D0DB
:105AA00024E0286840F480302860606888B1FDF701
:105AB000DFFB064609E0286840F480202860F0E714
:105AC000FDF7D6FB801B64287ED828688003F7D5B5
:105AD0000CE0FDF7CDFB064605E000BFFDF7C8FB77
:105AE000801B6428F0D828688003F7D420788007CA
:105AF00056D5D8F80000DFF85093396810F0380018
:105B0000A9F10C090ED0182801D188070AD0E06845
:105B1000A8B3296821F0190101432960FDF7A8FB0A
:105B2000064628E02868400702D5E06800288AD0A9
:105B3000E168286820F0190008432860FDF798FB09
:105B4000064606E0D2E000BFFDF792FB801B02286C
:105B5000BAD828684007F7D5217CD9F8002022F070
:105B6000FE4242EA0161C9F8001019E0FDF780FB2E
:105B7000801B0228A8D828684007F7D5ECE7FFE784
:105B8000286820F001002860FDF772FB064604E05B
:105B9000FDF76EFB801B022896D828684007F7D4D3
:105BA0002078C00646D5D8F80000DFF89C92396806
:105BB00000F03800A9F10409082812D0182805D1EE
:105BC00001F00300012800E0CEE00AD0E0690028DF
:105BD000286820D040F080002860FDF749FB064689
:105BE00015E02868C00502D5E06980287ED194F8C8
:105BF0002010D9F8002022F07C5242EA0161C9F855
:105C0000001017E0FDF734FB801B0228A0D828689D
:105C1000C005F7D5EBE720F080002860FDF728FBF2
:105C2000064604E0FDF724FB801B022890D8286874
:105C3000C005F7D42078000729D58348616964300E
:105C400000298146016811D041F001010160FDF792
:105C50000FFB064605E000BFFDF70AFB801B02288C
:105C600088D8D9F800008007F6D510E021F00101AE
:105C70000160FDF7FDFA064605E000BFFDF7F8FA02
:105C8000801B022870D8D9F800008007F6D420784D
:105C9000800623D5A0690028286810D040F48050E1
:105CA0002860FDF7E5FA064605E000BFFDF7E0FADB
:105CB000801B022858D828688004F7D50EE020F40D
:105CC00080502860FDF7D4FA064604E0FDF7D0FACC
:105CD000801B022848D828688004F7D42078400721
:105CE00051D5DFF86891D9F8001000E015E141F4D2
:105CF0008071C9F80010FDF7BBFA064605E000BF49
:105D0000FDF7B6FA801B64282ED8D9F80000C0052C
:105D1000F6D54D4EA068603601280AD008B1052896
:105D200013D0306820F001003060306820F00400AB
:105D300002E0306840F001003060A06841F2883A2B
:105D400098B1FDF795FA81460AE0306840F004000A
:105D50003060EEE7FDF78CFAA0EB0901514503D85E
:105D600030688007F6D50EE072E0FDF781FA8146D3
:105D700006E000BFFDF77CFAA0EB0901514567D8AA
:105D800030688007F6D4606A00287CD0DFF8B8A0BD
:105D9000D8F800100AF1200A4FF6F87B0AF104083F
:105DA000C1F3C2010329AAF104096DD002282868B1
:105DB00020F08070286003D0FDF75AFA044681E095
:105DC000FDF756FA064604E0FDF752FA801B02285A
:105DD00075D828688001F7D4E26A40F2F331386858
:105DE00054F8283F884340EA021018433860217B6A
:105DF0004FF4FE0C22894FF0FE47208A4902267D8F
:105E0000521E401EA1F5007189B2C2F3080211436F
:105E1000761E0CEA00400143484607EA0662114339
:105E2000CAF80010D9F8001021F00101C9F80010DB
:105E3000D8F80030266A23EA0B0343EAC601C8F803
:105E40000010D9F8001004E010440258004802582D
:105E500035E0A26921F00C011143C9F80010016876
:105E6000E26921F0020111430160016841F48031CF
:105E70000160016841F400310160016841F4802152
:105E80000160016801E06CE020E041F00101016087
:105E9000286840F080702860FDF7EAF9044604E0C5
:105EA000FDF7E6F9001B022809D828688001F7D51C
:105EB00057E000BFFDF7DCF9001B022802D90320E0
:105EC000BDE8F09F28688001F4D44AE039680128D1
:105ED000DAF8000021D0A26A01F0030393421CD13A
:105EE000E26AC1F305118A4217D1216BC0F308029F
:105EF000491E8A4211D1616BC0F34622491E91426C
:105F00000BD1A16BC0F30642491E914205D1E16B52
:105F1000C0F30660491E814201D00120D0E7A16C88
:105F20004646D8F80000C0F3CC00814219D0D9F819
:105F300000004D4620F00100C9F80000FDF798F977
:105F40004FEA0007FDF794F9B842FBD0A26C306825
:105F500020EA0B0040EAC2003060286840F00100EF
:105F600028600020ACE700002DE9F04104001D4648
:105F700016460F4603D0D4F8880018B108E0012077
:105F8000BDE8F081002084F88400204600F09AFFEC
:105F90002420C4F888002068016821F00101016014
:105FA000A06A10B1204602F08BFB204602F074FC80
:105FB0000128E5D0206871050D4A41EA0541836852
:105FC00043F4804383602068836823F400433B43A9
:105FD00083602068036813400B43036020680168F6
:105FE00041F0010101602046BDE8F04102F0CCBB68
:105FF000FFFF00FC2DE9F047040029D0594A4FF07B
:1060000000092068584B594D9042C4F8289006D09A
:10601000984204D0A84202D0E1680F2918D8E1685C
:106020004FF0010AE76B0831C9080AEB57167143B4
:10603000904205D0984203D0A84201D0082907D841
:10604000904203D0984201D0A84204D1102902D92D
:106050000120BDE8F08794F8810020B9204684F83B
:10606000809000F085F8022084F8810020680168A3
:1060700021F0010101602068A1698268B1F1806F9F
:1060800002F4F81110D16268B2F5800F01D01AB194
:106090000AE0A26B22B107E0A26BB2F1805F03D1EC
:1060A000026842F4805202606068400209D5E068EC
:1060B000072806D32068236D026822F480721A43F1
:1060C00003E02068026822F480720260A66AE06938
:1060D000E26B25683043E3680A4310431843A86025
:1060E000D4E90D02D4E90581636A25691843D4F81F
:1060F00020C00A43266810432843A56DD4E90172E5
:10610000D4E9123140EA080040EA0C003843084361
:10611000104318432843F060606868B920688168BC
:1061200021F4C05141F4006181602068816821F44C
:10613000C06141F4806181602068016D21F001013E
:1061400001656068400206D52068626DC16821F073
:1061500000411143C160C4F8849084F881A00020FC
:1061600077E700000030014000380040003C00406C
:106170002DE9F04FB5B0054614212EA8FAF79EFA86
:10618000B8216846FAF79AFA644902262868052772
:10619000614C002588424FF080094FF003084FF012
:1061A000080A36D1002117958014CDE90001684610
:1061B000FEF720FD08B1FAF7B2FC5748103001682D
:1061C00041F480510160006800F4805033902068F1
:1061D00040F008002060206800F00800339020683C
:1061E00040F00200206020682EA9CDE9305800F070
:1061F00002004446CDE932704948CDE92E96FCF7BD
:1062000023FF48482EA9CDE93054CDE92EA6329778
:106210003DE04549DFF814B188423DD10021179592
:106220008014CDE900016846FEF7E4FC08B1FAF7F6
:1062300076FC39480830016841F48041016000680B
:1062400000F480403390206840F004002060206813
:1062500000F004003390206840F0020020602068C5
:106260002EA9CDE9305800F00200339006204446B4
:10627000CDE92E0658463297FCF7E6FE4FF4005063
:106280003297CDE92E0627482EA9CDE93054FCF7E8
:10629000DBFE35B0BDE8F08F25498842F9D10020FA
:1062A0004FF480414FF0A0422B92CDE90010684698
:1062B000FEF7A0FC08B1FAF732FC17481430016869
:1062C00041F020010160006800F020003390206858
:1062D00040F001002060206800F001003390206849
:1062E00040F00400206020682EA9CDF8B89000F09E
:1062F0000400CDE92F653195CDE932A00D48FCF7BA
:10630000A3FE4FF480502E90CDE92F65CDE9315793
:106310002EA95846BBE70000E04402580030014077
:10632000000C0258000402580038004000080258CF
:106330000014005800000258024A136883430B43BC
:10634000136070470404005870477047704700009E
:10635000F0B590F83C20012A43D0012280F83C207F
:10636000D1E90242204ECD6922F440722243D1E9A4
:10637000004322F480621A4322F400622243D1E9EE
:10638000043422F480521A430B6B22F4005222434D
:106390000C8B22F480421A43036822F4702242EAF2
:1063A0000442002422F08052B34242EA050202D0A5
:1063B0000E4DAB4210D10F8D22F4700CD1E9086262
:1063C000CD6A4CEA075121F08071314321F0007110
:1063D000114321F000522A435A6480F83C400020C7
:1063E000F0BD0220F0BD00000000014000040140AB
:1063F000F0B590F83C20012A41D0224E012480F8CB
:106400003C40022280F83D2002681F4D5368B24292
:10641000D2F808C001D0AA4203D14F6823F4700318
:106420003B430F6823F070031F4357600268B2427A
:1064300019D0B2F1804F16D0144B9A4213D0144B9E
:106440009A4210D0134B9A420DD0AA420BD0124B55
:106450009A4208D0114B9A4205D0114B9A4202D071
:10646000104B9A4204D189682CF080031943916043
:10647000002180F83D4080F83C100846F0BD022025
:10648000F0BD000000000140000401400004004095
:1064900000080040000C004000180040004001408F
:1064A00000E0004000E4004010B5040003D094F880
:1064B0003D0010B107E0012010BD002084F83C0031
:1064C000204600F022F8022084F83D002068211DBB
:1064D00001F0C4FE012084F8480084F83E0084F8EE
:1064E0003F0084F8400084F8410084F8420084F8BA
:1064F000430084F8440084F8450084F8460084F89A
:10650000470084F83D00002010BD704790F83D1012
:10651000012901D0012070471A4A022180F83D105C
:106520000168CB6843F00103CB60006890421AD049
:10653000B0F1804F17D01449884214D013498842D3
:1065400011D0134988420ED0124988420BD012490B
:10655000884208D01149884205D01149884202D0AA
:106560001049884207D181680F4A1140062906D098
:10657000B1F5803F03D0016841F0010101600020C6
:106580007047000000000140000400400008004087
:10659000000C004000040140001800400040014091
:1065A00000E0004000E400400700010070472DE9D2
:1065B000F041044600680027C6680569A90713D59D
:1065C000B10711D5FA1E0261012121772068806987
:1065D0008007204602D0FFF7E9FF04E000F0F8F85A
:1065E000204600F0EDF92777680716D5700714D517
:1065F000226802206FF00401116120772068806911
:1066000010F4407F204602D0FFF7D0FF04E000F0F6
:10661000DFF8204600F0D4F92777280715D5300792
:1066200013D5226804206FF00801116120772068DB
:10663000C0698007204602D0FFF7B8FF04E000F0F1
:10664000C7F8204600F0BCF92777E80616D5F00613
:1066500014D5226808206FF010011161207720689E
:10666000C06910F4407F204602D0FFF79FFF04E08E
:1066700000F0AEF8204600F0A3F92777E80708D02D
:10668000F00706D021686FF001000861204600F095
:1066900099F9280601D4A80408D5300606D5216842
:1066A0006FF4025008612046FFF74FFEE80508D559
:1066B000300606D521686FF4807008612046FFF728
:1066C00043FE680608D5700606D521686FF04000C5
:1066D0000861204600F080F9A8060AD5B00608D562
:1066E00021686FF0200008612046BDE8F041FFF707
:1066F0002DBEBDE8F081000030B587B004461421FE
:106700006846F9F7DBFF246800222B4D0223294954
:106710000120AC4211D10C6844F010040C600968EF
:1067200001F0100105914FF408510091CDE90132BB
:10673000CDE903202148694625E0B4F1804F12D00D
:106740001F4D2048AC4222D10C6844F002040C607A
:106750000968009301F00201CDE901320392CDE90D
:10676000043169460FE00C6844F001040C600968CC
:1067700001F00101059105210091CDE90132CDE93A
:10678000032011486946FCF75FFC07B030BD0F4D90
:10679000AC42FAD10C6844F002040C60096801F0C4
:1067A00002010591E9130091CDE90132CDE90323FE
:1067B0006946E8E7E0440258000001400010025832
:1067C0000004004000040258000002580018004075
:1067D000704770B5044690F83C0000260D4601282D
:1067E0000BD0012084F83C000C2A4AD007DC82B18F
:1067F000042A20D0082A06D131E0022070BD102AD8
:1068000053D0142A63D00126002084F83C0030467F
:1068100070BD206801F092FD2068816941F0080197
:1068200081612068816921F00401816120682A6901
:106830008169114311E0206801F0D2FD206881696F
:1068400041F4006181612068816921F48061816186
:1068500020682969826942EA01218161D4E72068C0
:1068600001F00AFE2068C16941F00801C161206899
:10687000C16921F00401C16120682A69C16911431D
:1068800011E0206801F044FE2068C16941F4006114
:10689000C1612068C16921F48061C16120682969F2
:1068A000C26942EA0121C161AEE7206801F06CFED5
:1068B0002068416D41F0080141652068416D21F07B
:1068C0000401416520682A69416D114311E0206887
:1068D00001F094FE2068416D41F40061416520683B
:1068E000416D21F48061416520682969426D42EA69
:1068F0000121416588E710B5040003D094F83D00FC
:1069000010B107E0012010BD002084F83C002046B3
:1069100000F022F8022084F83D002068211D01F0DB
:106920009DFC012084F8480084F83E0084F83F0074
:1069300084F8400084F8410084F8420084F8430061
:1069400084F8440084F8450084F8460084F8470041
:1069500084F83D00002010BD08B50168134881424D
:1069600001D113480FE01348B1F1804F0BD0124A08
:10697000914210D1016841F002010160006800F00D
:106980000200009008BD016841F00101016000684B
:1069900000F00100F5E7094A9142F3D1016841F0A6
:1069A00040010160006800F04000EAE7000001409B
:1069B000F0440258E8440258000400400018004027
:1069C0007047000000680349884201D1FCF756BCBB
:1069D0007047000000E00040704730B590F8841028
:1069E000012918D0012280F884202421C0F88810C1
:1069F0000022202401680B680D6823F0005325F065
:106A000001050D60426601680B60C0F8884080F89F
:106A10008420104630BD022030BD7047704770B5ED
:106A2000044690F8840001281DD0012284F88420B7
:106A30002420C4F8880020680568026822F001025A
:106A400002602068826822F060620A438260204609
:106A500001F014FE2268202100201560C4F888107F
:106A600084F8840070BD022070BD70B5044690F8B3
:106A7000840001281DD0012284F884202420C4F839
:106A8000880020680568026822F001020260206820
:106A9000826822F060420A438260204601F0EEFDE7
:106AA0002268202100201560C4F8881084F8840032
:106AB00070BD022070BD7047704770472DE9F041EE
:106AC00007680025044640F60F030226F869396876
:106AD000BA6818420AD183067ED501F0200302F07D
:106AE000805C53EA0C0377D0616F7EE1D44BDFF812
:106AF00054C3134001EA0C0C53EA0C0C6CD05FEA4F
:106B0000C07C0CD05FEAC15C09D54FF0010CC7F81E
:106B100020C0D4F8907047F00107C4F89070870740
:106B200009D5D70707D027683E62D4F8906046F0B1
:106B30000406C4F8906046070AD5D60708D027682F
:106B400004263E62D4F8906046F00206C4F89060D5
:106B500006070CD501F020061E4308D0266808233E
:106B60003362D4F8903043F00803C4F89030030542
:106B70000BD54B0109D526684FF400633362D4F876
:106B8000903043F02003C4F89030D4F89030002BBC
:106B90003DD0800609D501F0200002F08051084365
:106BA00003D0616F09B1204688472168D4F890006E
:106BB0008968490602D410F0280F2AD0204601F037
:106BC00041FE2068806840061ED52068083050E8E5
:106BD000001F21F0400100E021E040E80012002AFF
:106BE000F3D1D4F8800078B197490165D4F88000DA
:106BF000FAF7DAFF00280AD0D4F88000016D00E02F
:106C00002046BDE8F04108472046FFF756FFBDE8A3
:106C1000F0812046FFF751FFC4F89050F7E7D4F811
:106C20006CC02023BCF1010F7ED15FEAC06C7BD524
:106C30005FEAC16C78D51020386220688068400611
:106C400073D5D4F8802081491068884234D07F49B8
:106C50001831884230D07D49303188422CD07B4970
:106C60004831884228D079496031884224D0774918
:106C70007831884220D07549903188421CD07349C0
:106C8000A831884218D07249884215D0704918310D
:106C9000884211D06E49303188420DD06C4948315C
:106CA000884209D06A496031884205D06849783104
:106CB000884201D06649903140684FF480770004E3
:106CC000000C40D0B4F85C1081423CD9A4F85E00BE
:106CD000D069B8422FD0216851E8000F20F48070AD
:106CE00041E80002002AF6D12068083050E8001F71
:106CF00021F0010140E80012002AF5D12068083097
:106D000050E8001F21F0400140E80012002AF5D1B0
:106D1000C4F88C30E566206850E8001F21F01001AF
:106D200040E80012002A01E04AE019E0F3D1D4F86B
:106D30008000FAF789FD2667B4F85C00B4F85E10AD
:106D4000401A81B208E0B4F85C1081427FF466AF6B
:106D5000D069B842FAD126672046FFF75EFE56E7B3
:106D6000B4F85C00B4F85E10B4F85E20401A81B24A
:106D7000002AF4D00029F2D0226852E8000F20F453
:106D8000907042E80007002FF6D1324F206800F1E2
:106D9000080050E8002F02EA070240E8002CBCF18E
:106DA000000FF3D1C4F88C30E5666567226852E8BD
:106DB000000F20F0100042E80003002BF6D1CAE7D4
:106DC000C60209D5560207D54FF480103862204616
:106DD000BDE8F041FFF770BE06060AD501F0800657
:106DE00002F40002164304D0A16F00297FF408AF1B
:106DF0000DE7420611D54A060FD52046016851E835
:106E0000002F22F0400241E80024002CF6D1C0F807
:106E10008830856700F0A2F9F9E6020206D54A003B
:106E200004D52046BDE8F041FFF745BEC00196D528
:106E3000002994DA2046BDE8F041FFF7EFBD0000DD
:106E400001000010200100043388000810000240F7
:106E500010040240FEFFFFEF10B5040003D0D4F889
:106E6000880010B107E0012010BD002084F88400E4
:106E7000204600F027F82420C4F888002068016824
:106E800021F001010160A06A10B1204601F018FC58
:106E9000204601F001FD0128E6D02068416821F478
:106EA000904141602068816821F02A01816020685A
:106EB000016841F0010101602046BDE8104001F089
:106EC00063BC00002DE9F04FB5B0804614212EA818
:106ED000F9F7F4FBB8216846F9F7F0FB944C022669
:106EE00095490727D8F80000083C914D4FF000085D
:106EF000DFF840A288422DD10020CDF87480022115
:106F0000CDE900106846FDF775FE08B1F9F707FEF8
:106F1000286840F080402860286800F08040339066
:106F2000206840F01000206020684FF4C0712E915E
:106F30002EA900F010003390CDE92F68CDE93187FC
:106F40005046FCF781F8002205215220FCF72EFA6A
:106F5000522033E07949DFF8E891884233D10020AC
:106F6000CDF878800121CDE900106846FDF742FE9A
:106F700008B1F9F7D4FDD9F8001041F01001C9F8B3
:106F80000010D9F8000000F010003390206840F0A5
:106F90000100206020682EA900F0010033904FF41A
:106FA000C06081E841016748CDE93187FCF74CF8C2
:106FB000002205212520FCF7F9F92520FCF7E8F946
:106FC00035B0BDE8F08F6049DFF880B188422CD140
:106FD0000020CDF874800221CDE900106846FDF74D
:106FE00009FE08B1F9F79BFD286840F400302860DD
:106FF000286800F400303390206840F008002060DA
:10700000206870212E912EA900F008003390CDE960
:107010002F68CDE931875846FCF716F80022052184
:107020002620FCF7C3F92620C8E74949884241D108
:107030000020CDF874800222CDE900206846FDF7DB
:10704000D9FD08B1F9F76BFD286840F4802028606D
:10705000286800F480203390206840F0020020600F
:10706000206800F002003390206840F008002060A3
:1070700020682EA9444600F0080033904FF4804069
:107080002E90CDE92F683348CDE93187FBF7DCFF3F
:107090004FF440702E90CDE92F64CDE931472EA9F1
:1070A0005846FBF7D1FF002205212720FCF77EF987
:1070B000272083E72849884282D10020CDF87880B4
:1070C0000121CDE900106846FDF794FD08B1F9F7FC
:1070D00026FDD9F8001041F08001C9F80010D9F858
:1070E000000000F080003390206840F01000206025
:1070F00020682EA9544600F010003390042081E847
:107100004101CDE931805046FBF79EFF2EAA0820B1
:107110000B2182E84101CDE931812EA92046FBF700
:1071200093FF002205219C20FCF740F99C2045E7B5
:10713000E844025800100258007800400010014056
:10714000F04402580000025800440040000C02586D
:107150000048004000040258001C01407047FEE750
:10716000F0B500230A251C463026372711E000BF62
:10717000B5EB107F02D906EB107C01E007EB107C29
:1071800001F813C001EB430C00015B1C8CF80140BB
:10719000DBB29342ECD3F0BD00EB8100006E00F057
:1071A000F84070478068C0F3C00070478068C0F343
:1071B000800070478068C0F38000704700EB810159
:1071C000034B51F8600F20F00040104308607047F7
:1071D0000060025830B58DB000246846242109941F
:1071E0000A940B94F9F76AFA24480425224B4FF4C9
:1071F0001012012103600223C0E90124C0E9041533
:10720000047603224176C36180F820408462C0E99D
:107210000B42C463046480F844408164FAF746F981
:1072200008B1F9F77CFC154809A90994F9F790FD14
:1072300008B1F9F774FC1248062140F2FF7203927C
:107240008DE823000D486946CDE904548DF82140AE
:10725000F9F712FE08B1F9F762FC0C210948CDE9F3
:10726000000106486946F9F707FE002801D0F9F742
:1072700056FC0DB030BD000000200240C0000020D0
:107280001000C0100000B84F094808B5016841F06F
:107290000101016000680022052100F0010000905A
:1072A0000B20FCF783F8BDE808400B20FCF770B812
:1072B000D84402581748002170B5154D012281604D
:1072C000182605600225C16020240174042341743E
:1072D00081744661C0E90625026242628262C2622E
:1072E000C0E90C210464C0E90E21C0E91131C0E9F4
:1072F0001331C0E91531C0E91714C0E91913FBF7C0
:107300008DFC002803D0BDE87040F9F708BC70BDC3
:1073100000A00040A80100201848002170B5164DBB
:1073200001220560182581602024C16004230174B6
:1073300041748174C0E90552C26140F2064502629F
:1073400042628262C262C0E90C250464C0E90E2177
:10735000C0E91131C0E91331C0E91531C0E9171492
:10736000C0E91913FBF75AFC002803D0BDE87040B0
:10737000F9F7D5BB70BD000000A400404802002012
:107380001848002170B5164D01220560182581604E
:107390002024C1600423017441748174C0E9055242
:1073A000C26140F61205026242628262C262C0E9B4
:1073B0000C250464C0E90E21C0E91131C0E9133184
:1073C000C0E91531C0E91714C0E91913FBF726FC11
:1073D000002803D0BDE87040F9F7A1BB70BD0000E4
:1073E00000D40040E8020020044A0021044810B5FF
:1073F00003F0AAFA0349086010BD0000C8C00008E5
:10740000AB800008000000202DE9F04F87B0142168
:107410006846F9F753F95848016841F010010160D6
:10742000016801F010010591016841F0040101605B
:10743000016801F004010591016841F080010160DB
:10744000016801F080010591016841F001010160CE
:10745000016801F001010591016841F0020101603C
:10746000016801F002010591016841F00801016025
:1074700000680122DFF804B14EF2290100F0080093
:1074800005905846FBF7EEFE4FF400463C480022BC
:107490003146FBF7E7FE4FF440683A480022414688
:1074A000FBF7E0FE4FF48059364801224946FBF7CE
:1074B000D9FE4FF4806A344800225146FBF7D2FED1
:1074C0000024694601254FF460400090CDE9015445
:1074D00058460394FBF7B8FD032769462920CDE9F8
:1074E0000005CDE902475846FBF7AEFD4FF4A0502A
:1074F00000904FF488106946CDE901042048FBF75D
:10750000A3FD00966946CDE901541D480394FBF79D
:107510009BFDCDF800806946CDE9015419480394DC
:10752000FBF792FD17486946CDE90095CDE9025772
:10753000FBF78AFDCDF800A06946CDE90154124859
:107540000394FBF781FD2802104D02218DE8130002
:107550006946284603940494FBF776FDCDE9006460
:10756000694628460294FBF76FFD0021A802FEF74A
:10757000E3FE07B0BDE8F08FE0440258000802586F
:107580000010025800040258000C02580000025873
:1075900070B586B018216846F9F790F818480822A7
:1075A000164D0021012417238160D606E0E803521E
:1075B000032580E81A0000F11403C0E9031483E8EE
:1075C00062000162C0E90912C16201630C48FCF764
:1075D0002FF908B1F9F7A3FA4FF0011041F2883200
:1075E00069460094CDE902400548FBF711FF0028E9
:1075F00001D0F9F794FA06B070BD000000A0005267
:10760000E00000242DE9F0414FF480051448134AAE
:1076100007276E114FF0007C2C0180E8E410002158
:10762000A300C0E90514C0E9073141629A008162F4
:10763000C162C0E90D21C163016441648164C16418
:10764000016541658165FEF7D5FC002803D0BDE8E2
:10765000F041F9F764BABDE8F08100000030014064
:107660003C0100242DE9F041164807264FF08042E6
:10767000DFF84CC00021551105611311C0E9021655
:10768000C0E907214162171281629411C162C0E909
:107690000D21C163016441648164C1640165416578
:1076A0008165C0E90543C0E900C7FEF7A3FC0028D7
:1076B00003D0BDE8F041F9F732BABDE8F08100002F
:1076C00000380040C40100242DE9F0414FF4800748
:1076D00015480021134EBD000722AC00C0E903216C
:1076E000A300C0E9073141629A0081624FF4003C77
:1076F000C162C0E90D21C163016441648164C16458
:10770000016541658165C0E9055480E8C010FEF758
:1077100071FC002803D0BDE8F041F9F700BABDE8DC
:10772000F0810000001400584C02002410B58AB00B
:10773000002468461C21079408940994F8F7BEFFBA
:10774000164840F2CF711722134BC0E90241046181
:107750008461C0E90032FFF7CEF808B1F9F7DFF92C
:107760000E4807A907940994FEF742FE08B1F9F7FD
:10777000D6F960206946CDE9000408480422029445
:107780000494FFF726F808B1F9F7C9F90348FEF7A2
:10779000B3FF0AB010BD0000001800406C040020C8
:1077A00010B598B000241C210DA8149415941694BB
:1077B000F8F784FF34216846F8F780FF274818223D
:1077C000254942F2107380E81600C0E90334446191
:1077D0008461FFF790F808B1F9F7A1F91F4814A9DF
:1077E000149415941694FEF703FE08B1F9F797F96F
:1077F0000DAA41F28831602082E813001748002268
:107800000DA91094119412941394FEF7E2FF08B19D
:10781000F9F785F9114808220DA9FEF7DAFF08B13A
:10782000F9F77DF94FF4005000940394010301949B
:10783000CDE904400294CDE9084108486946069420
:107840000A940C94FEF784FD08B1F9F768F903482F
:10785000FEF752FF18B010BD000001408803002061
:1078600010B58AB0002468461C2107940894099436
:10787000F8F724FF1A4842F2107118224FF08043A3
:10788000C0E9024104618461C0E90032FFF733F8C6
:1078900008B1F9F744F9124807A907940994FEF7CB
:1078A000A7FD08B1F9F73BF9602041F288318DE876
:1078B00013000B48002269460494FEF78AFF08B1C2
:1078C000F9F72DF9064808226946FEF782FF08B14C
:1078D000F9F725F90248FEF70FFF0AB010BD0000C6
:1078E000D403002030B58BB0002468461C210794D7
:1078F00008940994F8F7E2FE164842F20F72172333
:10790000134D8021C0E9024204618161C0E9005346
:10791000FEF7F1FF08B1F9F702F90E4807A907943D
:107920000994FEF765FD08B1F9F7F9F8602069469A
:10793000CDE9000407480C2202940494FEF749FFA5
:1079400008B1F9F7ECF80348FEF7D6FE0BB030BDEE
:1079500000040040200400201848002110B5164CF7
:107960000C224FF461230460C0E90131C160C0E919
:1079700004128161C161016241628162FFF76CFAA8
:1079800008B1F9F7CCF80D480021FFF76EF808B1FF
:10799000F9F7C5F809480021FFF741F808B1F9F7F0
:1079A000BEF80648FFF719F8002803D0BDE81040DC
:1079B000F9F7B5B810BD000000780040B804002009
:1079C0001848002110B5164C0C224FF461230460B6
:1079D000C0E90131C160C0E904128161C161016285
:1079E00041628162FFF738FA08B1F9F798F80D485B
:1079F0000021FFF73AF808B1F9F791F8094800219A
:107A0000FFF70DF808B1F9F78AF80648FEF7E5FF29
:107A1000002803D0BDE81040F9F781B810BD000080
:107A2000001C0140080700201848002110B5164C22
:107A30000C224FF461230460C0E90131C160C0E948
:107A400004128161C161016241628162FFF704FA3F
:107A500008B1F9F764F80D480021FFF706F808B1FE
:107A6000F9F75DF809480021FEF7D9FF08B1F9F7E9
:107A700056F80648FEF7B1FF002803D0BDE81040D5
:107A8000F9F74DB810BD0000001001404C05002072
:107A90001948002110B5174C4FF461230C220460E3
:107AA000C0E90131C1600B46C0E9041281610A4698
:107AB000C161016241628162FEF756FA08B1F9F7CD
:107AC0002EF80D480021FEF7D0FF08B1F9F727F88E
:107AD00009480021FEF7A3FF08B1F9F720F806488E
:107AE000FEF77BFF002803D0BDE81040F9F717B878
:107AF00010BD000000440040E005002019480021AE
:107B000010B5174C4FF461230C220460C0E9013119
:107B1000C1600B46C0E9041281610A46C16101627D
:107B200041628162FEF720FA08B1F8F7F8FF0D48CC
:107B30000021FEF79AFF08B1F8F7F1FF094800218C
:107B4000FEF76DFF08B1F8F7EAFF0648FEF745FFBC
:107B5000002803D0BDE81040F8F7E1BF10BD0000D9
:107B6000004800407406002010490122104810B55A
:107B700001F0EEFC08B1F8F7D2FF0E490C4801F015
:107B800006FF08B1F8F7CBFF0B49094801F0A2FA4C
:107B900008B1F8F7C4FF064801F07EFF08B1F8F716
:107BA000BEFFBDE81040FCF7D5BC00000400002477
:107BB000D40200248800002024000024FEE7FEE711
:107BC000F0B503004FF0000004460BD0022B09D89B
:107BD00041B100220A604A60022B8A60CA600A61D1
:107BE00002D007E00120F0BD294A1268D20734D044
:107BF0004FF40074274D002205EB8203D3F80434C0
:107C0000DE0707D003F0020604F00207BE4201D1EE
:107C1000561C0E60DE0607D503F0200604F0200790
:107C2000BE4201D1561C4E60DE0507D503F4007636
:107C300004F40077BE4201D1561C8E60DE0311D5DC
:107C400003F4802604F48027BE420BD19E0302F188
:107C5000010604D446F4803603E00F4CCAE746F030
:107C60008076CE60DE010FD503F0806604F0806779
:107C7000BE4209D19B0102F1010302D443F48033D7
:107C800001E043F080730B61521C022AB4D3F0BDB3
:107C900000B4005200B00052220204042DE9F04169
:107CA000984616460F460446069D08E0681C06D016
:107CB000FBF7DEFAA0EB0800A8420AD84DB1206815
:107CC000006A384000D00120B042EFD10020BDE86A
:107CD000F0814FF400702065606D40F00100606538
:107CE0000120F4E70148FCF72FB80000D00700247A
:107CF0002DE9F041044680790D46202723680128AC
:107D00004FF4004604F29C4203EB4511D3F840C007
:107D1000D1F8080B09D0DFF89CE0F4453AD1020411
:107D200033D500BFC1F8086B40E0234B5FEA007E0B
:107D300004D59C453AD90004F4D437E05FEA806E5C
:107D400002D5C1F8087B31E010F0280F2ED19C45F8
:107D500001D90004E6D4D1F8101B05EBC50004EBF3
:107D60008000C1F31201D0F87432A3EB0101C0F816
:107D7000681200F51570ADB903691BB1C2681144F2
:107D8000C1600FE0206801210AE080060AD5C1F831
:107D9000087B07E035B9D4F8640218B90021184609
:107DA00002F0FAF92046E9B2FBF7B7FE0020BDE881
:107DB000F08100000A31544F0A30544F2DE9F84F3A
:107DC0000E460568814601EBC60100EB8104D4E94B
:107DD00009201434904202D90120BDE8F88FA1682F
:107DE000101A814200D20846C01C05EB46188708CD
:107DF0001BE000BFA268A0EB010A524500D29246E8
:107E000099F806100AF1030000911FFA8AF3E1685D
:107E100087082846F2B202F003FDE16801EB0A0090
:107E2000E060616901EB0A006061D8F8180980B26E
:107E3000B84205D3D4E90401814201D20028D9D146
:107E4000D4E90401884208D8D5F83418012006F096
:107E50000F0290408143C5F834180020BDE70000B0
:107E60002DE9F047454D044689464FF0000A286841
:107E7000C04380070AD0414E283E306820F0806021
:107E80003060FBF7F5F90746B04608E00120BDE891
:107E9000F08700BFFBF7ECF9C01B022867D8D8F8C1
:107EA00000000001F6D4206829684FF4FE0721F491
:107EB0007C313E0241EA00302860207AA389B4F880
:107EC00004C040022D4D2D495B1E227CACF1010CFB
:107ED0001035091DA0F5007080B2521ECCF3080CBD
:107EE00007EA034340EA0C00184306EA0262104323
:107EF00028600868626920F0C000104308600A68C2
:107F0000A06922F0200202430A60281D0A6822F0BC
:107F100010020A6002684FF6F873E4699A4342EA75
:107F2000C40202600868B9F1000F40F010020A6054
:107F300011D00868B9F1010F11D040F400100860A9
:107F4000D8F80000444640F08060C8F80000FBF715
:107F50008FF905460DE0086840F40020EFE740F493
:107F60008010ECE7FBF784F9401B022801D90320BD
:107F70008DE720680001F5D5504688E7284402586F
:107F80002DE9F047454D044689464FF0000A286820
:107F9000C04380070AD0414E283E306820F0805010
:107FA0003060FBF765F90746B04608E00120BDE800
:107FB000F08700BFFBF75CF9C01B022867D8D8F830
:107FC00000008000F6D4208829684FF4FE0721F0D5
:107FD0007C713E0241EA00502860207AA389B4F8FF
:107FE00004C040022D4D2D495B1E227CACF1010CDA
:107FF0001835091DA0F5007080B2521ECCF3080C94
:1080000007EA034340EA0C00184306EA0262104301
:1080100028600868626920F44060104308600A68BC
:10802000A06922F4007202430A60281D0A6822F443
:1080300080720A6002684FF6F873E4699A4342EA74
:10804000C40202600868B9F1000F40F480720A604F
:1080500011D00868B9F1010F11D040F080700860AC
:10806000D8F80000444640F08050C8F80000FBF704
:10807000FFF805460DE0086840F48000EFE740F4A3
:108080000000ECE7FBF7F4F8401B022801D90320BD
:108090008DE720688000F5D5504688E728440258CF
:1080A0000178407841EA00207047FFF75DFD01202C
:1080B00002F00DFCFBE74FF0E02010B5006903F083
:1080C00049FE012803D0BDE8104003F06DBB10BD90
:1080D00070B59CB04C216846F8F7F0FA202113A83F
:1080E000F8F7ECFA0220FCF70BFA2248016821F4B9
:1080F000404101600168002401F440411B91016886
:108100008904FCD502204025C30323220121CDE9A7
:108110000023CDE9031528220990069104230D912F
:108120000C260A90CDE90B02CDE90E30CDE91064A2
:1081300068461294FDF784FC08B172B6FEE7082287
:108140001A95CDE91625D30113AA3F200321CDE9C5
:10815000185382E8130013A8FDF7EAF908B172B6C4
:10816000FEE700214FF480220846FDF71FFC1CB0FB
:1081700070BD0000184802582D48F0B52D4A01681E
:1081800041F470010160106800F00F00072804D26C
:10819000106820F00F00C01D106027490020264CF9
:1081A00010340B68254D43F001030B6020600B6811
:1081B0002B400B60136803F00F03072B04D91368DF
:1081C00023F00F03DB1D13601B4C1D4A18341D4B9D
:1081D000261D371D2060184C1B4D28343060261D8D
:1081E0003860371D23603B1D35601C1D3A60251D1E
:1081F0002E1D1860331D22602860326018600B68E5
:108200000D4A0D4C23F48023D4320B60603420607F
:108210001068C0040BD4136843F2D2000B4943F436
:10822000805313600860106820F480501060F0BD27
:1082300088ED00E000200052004402587FEDF6EA8D
:1082400080020101000202020000FF010040005212
:108250000148FEF7ACB900009C0700202DE9F0476B
:108260002C4B4FF0804A2C4D026898422B4E2C4FDD
:108270002C4C09D0504507D0A84205D0B04203D0BD
:10828000B84201D0A04205D1D1F804C022F070025A
:108290004CEA0202DFF890C0DFF890809842DFF8E5
:1082A000909015D0504513D0A84211D0B0420FD0B5
:1082B000B8420DD0A0420BD0604509D0404507D050
:1082C000484505D01B4DA84202D01B4DA84203D102
:1082D000CD6822F440722A438E684D6922F08002F4
:1082E000C6620E682A439842866207D0A04205D033
:1082F000604503D0404501D0484501D1096901637B
:108300000368012143F00403036041610260BDE89A
:10831000F087000000000140000400400008004019
:10832000000C0040000401400040014000440140B6
:108330000048014000E0004000E400402DE9F04F1B
:10834000DFF88480214EDFF88890DFF888B0026A79
:10835000036AB042DFF880A022F0020C1F4F23F026
:1083600001020262426885698B680C6805EA0805AB
:1083700025F0030543EA0C0344EA050407D0484509
:1083800005D0584503D0504501D0B84205D1CD683D
:1083900023F008031D4325F00403B04207D04845ED
:1083A00005D0584503D0504501D0B84205D122F43C
:1083B0004076D1E9055235432A43426084614968D9
:1083C00041630362BDE8F08F8FFFFEFF00000140B4
:1083D00000040140004001400044014000480140C9
:1083E000F0B5DFF87CE01F4C1F4D026A036AA04223
:1083F00022F0200623F01003036242688369D1F85B
:1084000008C00F6803EA0E0323F4407E46EA0C130B
:108410004EEA072601D0A84206D1CF6823F0800398
:1084200043EA071323F04003A0420AD0A84208D031
:108430000E4CA04205D00E4CA04202D00D4CA042E2
:1084400007D1D1E9054522F4406242EA840242EABA
:10845000850242608661496881630362F0BD000065
:10846000FF8FFFFE0000014000040140004001407A
:108470000044014000480140F0B5DFF87CE01F4DAA
:108480001F4E026A036AA84222F4007723F4807325
:1084900003624368C269D1F808C002EA0E020C68A0
:1084A00022F0030E47EA0C2244EA0E0401D0B04247
:1084B00006D1CF6822F4006242EA072222F48062E9
:1084C000A8420AD0B04208D00E4DA84205D00E4DA9
:1084D000A84202D00D4DA84207D1D1E9055623F498
:1084E000405343EA051343EA06134360C4614968F5
:1084F000C1630262F0BD00008FFFFEFF000001407B
:108500000004014000400140004401400048014097
:10851000F0B5046A026A22F4805202624268C369BA
:1085200024F40054DFF848C08E680D6803EA0C0399
:10853000104F23F4407344EA0634B84243EA05235B
:108540000BD00D4DA84208D00C4DA84205D00C4DC3
:10855000A84202D00B4DA84204D14D6922F48042BA
:1085600042EA85124260C361496801640462F0BD59
:10857000FF8FFFFE00000140000401400040014069
:108580000044014000480140F0B5164F164B026A06
:10859000046A984222F4003524F48033036242686E
:1085A000436D0E890C6803EA070344EA030445EAB5
:1085B00006430BD00D4DA84208D00D4DA84205D062
:1085C0000C4DA84202D00C4DA84204D14D6922F4B2
:1085D000803242EA0522426044654968816503624F
:1085E000F0BD00008FFFFEFF0000014000040140CD
:1085F000004001400044014000480140F0B5164FE2
:10860000164B026A046A984224F48013036222F42F
:1086100000144268436D0E890D6803EA070344EABB
:10862000065443EA05230BD00D4DA84208D00D4D4A
:10863000A84205D00C4DA84202D00C4DA84204D14E
:108640004D6922F4802242EA8522426043654968EE
:10865000C1650462F0BD0000FF8FFFFE0000014015
:108660000004014000400140004401400048014036
:108670000148FEF723BA0000B804002030B5416E6F
:10868000B9B101680D4B03F108048A688968C2F327
:108690004262490F5D5C615C2D01B5FBF1F1A0F810
:1086A0006A10995CA25C0901B1FBF2F1A0F86810B4
:1086B00030BD0121A0F86A10F8E7000068C1000889
:1086C00090F82810090706D50168836B4A6822F4E0
:1086D00000421A434A6090F82810C90706D0016882
:1086E000C36A4A6822F400321A434A6090F828109C
:1086F000890706D50168036B4A6822F480321A4361
:108700004A6090F82810490706D50168436B4A680B
:1087100022F480221A434A6090F82810C90606D530
:108720000168C36B8A6822F480521A438A6090F809
:108730002810890606D50168036C8A6822F4005265
:108740001A438A6090F82810490611D50168436CD5
:108750004A6822F480121A434A60416CB1F5801FC6
:1087600006D10168836C4A6822F4C0021A434A6049
:1087700090F82810090606D50168C26C486820F4F4
:1087800000201043486070472DE9F8430025044657
:10879000C0F89050FAF76CFD8046206820266FF0F4
:1087A0007E470068000713D5002243463104204667
:1087B000009700F05FFA58B1216851E8000F20F0EF
:1087C000800041E80002002AF6D1C4F8886021E068
:1087D00020680068400722D5002243464FF48001FC
:1087E0002046009700F046FAC8B1206850E8001F04
:1087F00021F4907140E80012002AF6D12068083078
:1088000050E8001F21F0010140E80012002AF5D1D4
:10881000C4F88C60032084F88450BDE8F883C4F861
:108820008860C4F88C60E5662567002084F8845071
:10883000F3E710B5806B0021A0F85E10FEF73DF95C
:1088400010BD000010B5026852E8001F21F49071BD
:1088500042E80013002BF6D10E4B0268083252E8B2
:10886000001F194042E80014002CF6D1C16E012906
:1088700008D1026852E8001F21F0100142E80013FD
:10888000002BF6D100212022C0F88C20C166416760
:1088900010BD0000FEFFFFEF2DE9F04304468068A5
:1088A000E24E87B0E24B2168D4E90427D4F81CC01B
:1088B00010430A68002547EA0C0738433240024358
:1088C0000A602068E268416821F440511143416028
:1088D0002268A1699A4201D0206A01439668DFF8B4
:1088E00054C3D54FD54806EA0C060E43966021685E
:1088F000666ACA6A22F00F023243CA622268BA422A
:108900000ED1006800F0380018286FD07ADCB8B3B8
:1089100008286CD010286BD18BE0282868D18EE015
:10892000C7498A4209D1006800F0070006285FD2D3
:10893000DFE800F0507D7F818385C2498A4209D1FA
:10894000006800F0070006287BD2DFE800F04370E3
:1089500072747678BC498A4209D1006800F0070039
:1089600006286ED2DFE800F036636567696BB749A9
:108970008A420BD1006800F00700062861D200E0AF
:1089800043E0DFE800F0275456585A5CB0498A4269
:1089900006D1006800F0380018284CD0B7DD31E06F
:1089A000AC498A4209D1006800F00700062848D285
:1089B000DFE800F0103D3F414345A7498A420BD113
:1089C000006800F0070006283BD2DFE800F0033023
:1089D00032343638002035E0A0498A4209D1006897
:1089E00000F03800182826D091DD0BE023E01EE0CF
:1089F00027E09B498A420AD1006800F03800182815
:108A000019D084DD202888D11CE001201AE09A4288
:108A100017D18A48001D006800F00700062810D210
:108A2000DFE800F0030507090B0D02200AE004202F
:108A300008E0082006E0102004E0202002E04020AA
:108A400000E080208749DFF820829A42874A4FF46D
:108A500000434FEA21174FF000064ED110281AD0DC
:108A600006DC022809D004280BD008287ED10DE0AE
:108A700020283ED0402879D13DE0FBF773FD014628
:108A800010E06846FBF724FE01990BE003A8FBF712
:108A9000C1FE049906E01068800605D51068C0F391
:108AA000C100C140002970D0606A676838F81020A2
:108AB00007EB4703B1FBF2F0834257D8B0EB073F17
:108AC00054D8002308461946F7F702FD02467808F5
:108AD000130E120243EA012110183A467141002395
:108AE000F7F7F6FC624AA0F5407191423ED8216842
:108AF0008FE03946D8E71946D6E7D4F81CC04FF6C0
:108B0000EF799C4546D1082819D005DC58B10128D9
:108B10000CD0042875D10DE0102815D0202835D0B0
:108B200040286ED134E0FCF781FE01E0FCF790FEB6
:108B3000014610E06846FBF7CBFD01990BE003A866
:108B4000FBF768FE049906E01068800604D51068FB
:108B5000C0F3C100C140C1B1636A606838F8133026
:108B6000B1FBF3F1490001EB500100E049E0B1FB3A
:108B7000F0F0A0F11001494543D84FF6F073216899
:108B8000C0F342021840104343E043E03946E3E7B4
:108B90001946E1E7082819D005DC58B101280CD0A6
:108BA00004282ED10DE0102815D020282BD04028E5
:108BB00027D12AE0FCF73AFE01E0FCF749FE014626
:108BC00010E06846FBF784FD01990BE003A8FBF772
:108BD00021FE049906E01068800604D51068C0F3F1
:108BE000C100C140B1B1636A606838F81330B1FBAD
:108BF000F3F101EB5001B1FBF0F0A0F11001494598
:108C000005D9012506E03946EDE71946EBE721686D
:108C100080B2C8600120A4F86A00A4F86800284661
:108C20006667A66707B0BDE8F0830000F369FFCF71
:108C3000000C0058FFF4FF1100100140544402588A
:108C40000044004000480040004C004000500040FC
:108C50000014014000780040007C004000180140F2
:108C6000001C01400090D00350C10008004402588D
:108C7000FFFC0F002DE9F047994617460D460446C4
:108C8000089E4FF0000833E0701C31D0FAF7F0FA7C
:108C9000A0EB0900B04218D8BEB1206801684907AE
:108CA00026D5802D24D0402D22D0C169C943090783
:108CB0000DD4082505622046FFF7C4FDC4F8905086
:108CC000012084F88480BDE8F0870320FBE7C069B9
:108CD000C04300050CD421684FF4006008622046B0
:108CE000FFF7B0FD2021C4F8901084F88480ECE7F1
:108CF0002068C06935EA000004D00020B842C3D023
:108D00000020E0E70120F9E70148FDF7D7BE0000A9
:108D1000080700200148FDF7D1BE00004C050020E7
:108D20000148FDF7CBBE0000E00500200148FDF73B
:108D3000C5BE0000740600202DE9F0410C46D0F8B5
:108D4000D412D0F8C83200EB8101D1F8C01229B397
:108D500004F00F02002702EB820500EB8506B569DF
:108D60004DB102EBC20203EB8202D269B5FBF2F312
:108D700002FB1352A2B1C1F81472D0F8D42200EB56
:108D80008200D0F8C40203692BB1D1F8080201F5C2
:108D90000471224698470020BDE8F0810320FBE7DC
:108DA000002321461A46B76100F0D3FDF3E770B502
:108DB0000546D0F8D40205EB8000D0F8C04294B14B
:108DC000284600F0A0FCC4F80C02D5F8D40205EB4C
:108DD0008000D0F8C412D4F80402CA6804F5037104
:108DE0009047002070BD032070BD000070B5224D7B
:108DF0000446297800F0C8FB2878002600F00F0010
:108E000000EB800004EB800086842046697800F047
:108E1000BBFB687800F00F0000EB800004EB8000E3
:108E2000A0F864612046A97800F0AEFBA87800F0B5
:108E30000F0000EB800004EB80008684C684D4F829
:108E4000D40204EB8000D0F8C01299B1D0F8C4026B
:108E500040688047D4F8D40204EB8000D0F8C00208
:108E600000F09FFFD4F8D40204EB8000C0F8C06289
:108E7000C4F8BC62002070BD8C00002410B5D0F88E
:108E8000D41200EB8100D0F8C04284B1D0F8C412F3
:108E900059B194F80002FF2807D08B68214694F856
:108EA00001229847FF2084F80002002010BD032013
:108EB00010BD00000A210180004870479000002486
:108EC00070B5822106460D4800F06AFA0121054678
:108ED0000A4800F065FA81210446084800F060FA6B
:108EE0000DB11021A9714FF0400104B1A18000B172
:108EF000818043203080014870BD00009C00002428
:108F000070B5822106460D4800F04AFA0121054657
:108F10000A4800F045FA81210446084800F040FA6A
:108F20000DB11021A9714FF4007104B1A18000B1FD
:108F3000818043203080014870BD00009C000024E7
:108F400070B5822106460D4800F02AFA0121054637
:108F50000A4800F025FA81210446084800F020FA6A
:108F60000DB11021A9714FF0400104B1A18000B1F1
:108F7000818043203080014870BD00009C000024A7
:108F80002DE9F0474FF407750446284600F00AFF24
:108F900006004FF0000965D02946F7F78FFBD4F89B
:108FA000D40201273C4D4FF4007A4FF0100804EB37
:108FB0008000C0F8C062C4F8BC62207CF0B329789D
:108FC00040230222204600F00EFC2878402300F0C7
:108FD0000F0000EB800004EB800087840222697898
:108FE000204600F000FC697808230322204601F0A7
:108FF0000F0101EB810104EB8101A1F86471A978F3
:1090000001F00F0101EB810104EB8101A1F8268041
:10901000A97800F0E8FBA978C84601F00F0101EB40
:10902000810104EB81018F84C6F80492D4F8D40244
:1090300004EB8000D0F8C402006800E01AE006F5F6
:1090400001768047C6F81080C6F8148032687AB17D
:10905000207CF8B140236978204600F0D0FB002046
:10906000BDE8F087D4F8D41204EB8101C1F8C092B6
:109070000220F5E7297802225346204600F0B3FB90
:109080002878534600F00F0000EB800004EB8000CE
:109090008784A3E75346DEE78C00002410B5D0F8A0
:1090A000D41200EB8101D1F8C01259B1027C084CF6
:1090B000002AD1F8042207D04023617800F09FFBFA
:1090C000002010BD032010BD4FF40073F5E7000031
:1090D0008C00002439B1D0F8D42200EB8200C0F813
:1090E000C4120020704703207047D0F8D42200EB50
:1090F0008200D0F8C00218B1C0F8041200207047F6
:1091000003207047D0F8D43200EB8300D0F8C002BF
:1091100028B1C0F81022C0F80812002070470320C0
:1091200070472DE9FC410646D0F8D4020C460021D8
:1091300006EB80000D46D0F8C0728DF80010ADF837
:10914000041037B1217811F060022CD0202A48D1C8
:1091500002E00320BDE8FC81E288E2B109060BD5FC
:10916000D0F8C4023946836860789847E288072AB5
:1091700000D9072239462CE0607887F80002E088A1
:10918000402800D340203946C2B2304687F8012239
:1091900000F057F82AE0D0F8C40200222146836884
:1091A0006078984722E0607830B101281ED00A2804
:1091B00009D00B2815D110E096F89C02032810D195
:1091C000022201A905E096F89C02032809D1012298
:1091D0006946304600F04FF808E096F89C020328F4
:1091E00004D02146304600F021F803252846B1E797
:1091F00010B5D0F8B82200245268904700B103247B
:10920000204610BD002070470020704713460A46D4
:10921000002110B500F0F3FA002010BD13460A46F5
:10922000002110B500F095FB002010BD10B5802185
:10923000044600F06FFB2046BDE81040002100F01E
:1092400069BB10B5C0F858210323C0F89432C0F8A8
:109250005C2113460A46002100F0D1FA002010BD1F
:1092600010B50521C0F8941200231A46194600F0E3
:10927000C6FA002010BD10B582610223C0F89432F6
:10928000C26113460A46002100F063FB002010BDB6
:1092900010B50421C0F8941200231A46194600F0B4
:1092A00058FB002010BDF8B504460D460020ADF86F
:1092B00000004888010A062947D006DC01290FD0A2
:1092C000022912D0032962D11DE0072946D00F29B7
:1092D0005DD1D4F8B402C26920E0694690473BE012
:1092E000D4F8B412207C0A68F7E7207C0226002814
:1092F000D4F8B80205D0C16A68468847014646706E
:1093000036E0816AF8E7C0B2062840D2DFE800F014
:1093100003090D111519D4F8B4024268B2B3207CC8
:10932000DBE7D4F8B4028268F8E7D4F8B402C26884
:10933000F4E7D4F8B4020269F0E7D4F8B402426961
:10934000ECE7D4F8B4028269E8E7207CF0B9D4F8FD
:10935000B802416B68468847014609E0207CA8B9FD
:10936000D4F8B802016B6846884701460720487068
:10937000EA888AB1BDF8000040B1824200D90246B5
:109380002046ADF80020FFF776FFF8BDFFE729463D
:109390002046FFF74BFFF8E72046FFF779FFF4E799
:1093A00078B542880D460178002604468A4212D9D3
:1093B000ADF800100AE0694600F019F84178052977
:1093C00004D181780646A94205D000266188BDF8FF
:1093D00000209142EFD8304678BD002102E0491CC0
:1093E000401CC9B20278002AF9D1084670470A88A1
:1093F00003781A440A8001780844704770B5002841
:1094000016460D4620D00446FFF7E7FF022201462C
:10941000100202EB4101814204D82046FFF7DDFF34
:109420004000801C30803378032102202B70002202
:10943000697006E0431C2954D8B2411C641C2A54AC
:10944000C8B221780029F5D170BD01004FF00000AD
:1094500004D0012901D0022901D003207047012046
:109460007047000004A00A46024910B5FFF7C6FF86
:10947000004810BDE807002043444320436F6E6658
:10948000696700001220088000487047080000202B
:1094900004A00A46024910B5FFF7B0FF004810BD0E
:1094A000E807002043444320496E74657266616397
:1094B0006500000004200880004870470400002078
:1094C00004A00A46024910B5FFF798FF004810BDF6
:1094D000E807002053544D6963726F656C656374CF
:1094E000726F6E696373000004A00A46024910B5EA
:1094F000FFF784FF004810BDE807002053544D33A8
:1095000032205669727475616C20436F6D506F72B2
:109510007400000010B51A2008800B480A49083072
:10952000021F096800681468081809D00749082252
:10953000FDF716FE0549042220461031FDF710FE06
:109540000248801E10BD000000E8F11F2A00002024
:1095500078B10023C0F8B832C0F8C432C0F8D032B5
:1095600009B1C0F8B4120121027080F89C1200F019
:10957000CFB80320704710B5D0F8C802FAF70FFB38
:10958000BDE81040FFF761BF10B5D0F8C802FAF788
:10959000E1FABDE81040FFF758BF2DE9F04117464A
:1095A00004464FF0000521B194F89C02032842D0F4
:1095B0004CE0D4F8941204F11400022935D1D0E91A
:1095C00002639E4206D9F21A394682602046FFF7AE
:1095D00025FE0FE0B34214D14068984211D3D4F86D
:1095E000981288420DD2002220461146FFF716FE3F
:1095F000C4F8985200231A461946204600F0FFF896
:1096000013E094F89C02032808D1D4F8B802C1688A
:1096100021B1C4F8D452C168204688478021204631
:1096200000F078F92046FFF71BFE94F8A00268B11D
:1096300084F8A0520AE0D4F8B802426932B1C4F802
:10964000D452426920469047002800D10020BDE84E
:10965000F08170B5134604464FF0000221B194F832
:109660009C02032830D03AE0D4F8941204F5AA7092
:10967000032934D1D0E902518D420AD96A1A826095
:109680000846824200D3024619462046FFF7BEFD37
:1096900025E094F8AA0210F01F0003D0012802D0A0
:1096A000022800D0002294F89C02032808D1D4F8A4
:1096B000B802016921B1C4F8D42201692046884763
:1096C0002046FFF7E5FD0AE0D4F8B802836933B11C
:1096D000C4F8D422826920469047002800D1002097
:1096E00070BD0020704710B5D0F8B812012280F884
:1096F0009C22002429B103794A68D9B2904700B16D
:109700000324204610BDD0F8C802FAF775BA00004D
:1097100070B50178012929D115490925154C022375
:109720000022C1F8E004C0F8C81208460C600D71B0
:10973000CB718A714B728A72CA720A738A73CA7346
:109740000A74FAF7D3FD08B1F7F7E9F908484FF4BE
:109750000071FAF7AEF9064880220021FAF7ADF958
:10976000034801214FF4BA72FAF7A7F9002070BD3F
:10977000D007002400000440D0F8C82201F07F0088
:109780000B0600EBC00002EB800001D5807D704726
:1097900090F85602704710B5D0F8D42200EB820240
:1097A000D2F8B82222B190F89C32032B02D004E008
:1097B000032010BD126A02B19047002010BD10B501
:1097C000D0F8D42200EB8202D2F8B82222B190F86D
:1097D0009C32032B02D004E0032010BD526A02B178
:1097E0009047002010BD10B51C46D0F8C8021346A3
:1097F0002246FAF70AFABDE81040FFF726BE10B578
:10980000D0F8C802FAF732FABDE81040FFF71DBEE3
:109810002DE9F041044601250020D4F8B81206468F
:1098200084F89C52C4F894026060C4F8A40284F8DE
:10983000A00231B14A6822B100212046904700B110
:1098400003262046002240231146FFF7CCFF402785
:10985000A4F8645100223B4680212046C4F8607180
:10986000FFF7C1FFA58430462762BDE8F08190F87C
:109870009C12042903D190F89D1280F89C120020BC
:10988000704710B590F89C12032905D1D0F8B81292
:1098900011B1C96901B18847002010BD01740020D1
:1098A000704710B5D0F8C802FAF7D6FDBDE81040F1
:1098B000FFF7CBBD70B5044600F2AA20054600F0C4
:1098C00051F894F8AA020123B4F8B01210F01F0264
:1098D000C4F89432C4F898120AD0012A0ED0022A91
:1098E00012D000F080012046BDE8704000F012B8B0
:1098F00029462046BDE8704000F0D0B829462046F1
:10990000BDE8704000F013BA29462046BDE870401B
:1099100000F05BB910B5D0F8C802FAF7C1F9BDE89C
:109920001040FFF792BD10B5D0F8C802FAF7AEFDAF
:10993000BDE81040FFF789BD90F89C12042903D0C0
:1099400090F89C1280F89D12042180F89C1200204F
:10995000704710B5D0F8C802FAF7DBF9BDE810403F
:10996000FFF773BD70B5054608788C1C28704878E1
:1099700068702046FEF794FBA41C68802046FEF722
:109980008FFBA880A01CFEF78BFBE88070BD38B56C
:1099900004460020ADF80000A1B1C4F8B812D4F814
:1099A000D40204EB8000D0F8B802C16A19B168464D
:1099B0008847C4F8D002D4F8D802401CC4F8D802B2
:1099C000002038BD032038BDD0F8B8320246002050
:1099D000002B02D01B681046184770472DE9F04154
:1099E0002C4E0446887800258846C1B20129317082
:1099F00006D941462046FFF719FC0320BDE8F08157
:109A000094F89C02022702280CD003281DD041465E
:109A10002046FFF70BFC31782046FFF7E9FB0325D2
:109A20002846EBE789B320466160FFF7CDFF0500CC
:109A300004D041462046FFF7F9FB1DE02046FFF722
:109A400027FC032084F89C02EAE7C1B160688842E1
:109A50001BD0C1B22046FFF7CBFB317820466160B6
:109A6000FFF7B2FF050010D041462046FFF7DEFBAE
:109A700021792046FFF7BCFB84F89C72D0E7616037
:109A800084F89C722046FFF7B3FB2046FFF700FCEA
:109A9000C6E7000088000024FFF745BF2DE9F0412C
:109AA0000A784FF0000512F060020CD0202A01D095
:109AB000402A7DD1D0F8D42200EB8202D2F8B8221D
:109AC0009268904731E04B78002201260A2B6FD232
:109AD000DFE803F041666E586E08056E2D29FFF72A
:109AE000E2FB67E004468888D8B9C888C8B94888C6
:109AF000802816D294F89C2200F07F07032A10D009
:109B00003946204684F89E72FFF7CBFE2046FFF7C9
:109B1000BFFB1FB1022084F89C024BE084F89C62DA
:109B200048E0204644E0FFF759FF054642E0CB8875
:109B3000012B3DD190F89C32012B04D0022B02D096
:109B4000032B35D104E000F108018260012216E008
:109B50000122011D13E090F89C22012A03D0022A61
:109B600001D0032A24D1CA88022A21D1D0F8A41214
:109B7000C66009B10321C160022200F10C01FFF7A8
:109B80007AFB17E04A88012A02D0022A03D00FE0AC
:109B9000C0F8A46216E08988090A80F8A01211E0D2
:109BA00090F89C32012B08D0022B06D0032B04D056
:109BB000FFF73CFB2846BDE8F08149880129F9D12F
:109BC000C0F8A422FFF764FBF4E72DE9F0410A781E
:109BD0000E460979054612F060004FF00008CCB23D
:109BE0000BD0202801D040286AD121462846FFF713
:109BF00009FBFF2800D0D8B396E07078C8B30128DD
:109C000024D003285CD195F89C02022802D00328B6
:109C100056D10CE0002C53D0802C51D02146284640
:109C2000FFF778FE80212846FFF774FE7CE07088FD
:109C300040B93CB1802C05D0F08818B9214628469F
:109C4000FFF768FE2846FFF723FB6DE095F89C02BE
:109C50000228DFD0032863D1708880BB600603D060
:109C600021462846FFF787FC2846FFF711FBBCE793
:109C700000E00AE0C5F8D402D5F8B8028268F2B173
:109C800031462846904780464EE095F89C020027D2
:109C9000022802D0032843D113E00CB1802C3FD11D
:109CA000200604F07F0000EB800005EB800101D569
:109CB000143101E001F5AA7102220F602CE033E0BB
:109CC0002EE0200604F00F0000EB800005EB800082
:109CD00009D5808C20B304F07F0000EB800005EBF9
:109CE000800614360AE0B0F86401C8B104F07F00C1
:109CF00000EB800005EB800606F5AA764CB1802CBF
:109D000007D021462846FFF737FD10B1012030600B
:109D100000E03760022231462846FFF7ACFA03E044
:109D200031462846FFF782FA4046BDE8F08170B51B
:109D3000054608780E464FF0000410F0600003D08E
:109D4000202801D0402827D195F89C02012803D073
:109D5000022801D003281FD1B088C1B201291AD826
:109D6000C1B22846FFF750FAFF280CD058B9D5F8F1
:109D7000B8128A683AB1C5F8D40228468A683146D2
:109D80009047044600E00324F088204307D128468A
:109D9000FFF77EFA03E031462846FFF747FA2046F0
:109DA00070BD704700487047B005002470B54D780D
:109DB00001230A78012D1C4C02F00F0503FA05F36C
:109DC000D0F81C5817D000EB421245EA0343C0F804
:109DD0001C38D2F8000B00040BD40B890979D2F897
:109DE000000BC3F30A03184344EA81410843C2F855
:109DF000000B002070BD9EB23543C0F81C5800EB2C
:109E00004213D3F800090004F3D40D890979D3F87B
:109E10000009C5F30A058904284341EA8251084331
:109E20002043C3F80009E4E700800010D0F80019CF
:109E30006FF30A01C0F80019D0F8041841F48071DA
:109E4000C0F804180020704770B50D460446C2F3F0
:109E500007211E460498012922D0E06840F0400006
:109E6000E060204600F03CF8C6F307210029A16B12
:109E70002ED021F48031A163C5F3074101290ED111
:109E8000E16D154A89B2E165E16D1143E165A168B3
:109E900041F00601A160A16841F02001A16070BD00
:109EA000A26BC3B20D49012B22F48030A063E0689D
:109EB00000EA0100E060E06820F44010E06003D1B7
:109EC000E06840F48010E060204600F009F8D3E735
:109ED00041F48031CFE700000000EE03BFFFBDFF7B
:109EE00008B500214FF070620091009B5B1C00934D
:109EF00093420CD80369002BF7DA0091016941F015
:109F0000010101610099491C0091914201D903208E
:109F100008BD0169C907F5D1002008BD70B50A78F0
:109F200001234C78012C00EB42122CD0D2F8004BCC
:109F3000002C0BDAD2F8004B44F00064C2F8004B5E
:109F4000D2F8004B44F08044C2F8004B0C78D0F8B3
:109F50003C5804F00F0403FA04F425EA0444C0F862
:109F60003C480978D0F81C4801F00F018B401C498F
:109F700024EA0343C0F81C38D2F8000B0840C2F8AA
:109F8000000B002070BDD2F80049002C0BDAD2F88B
:109F9000004944F00064C2F80049D2F8004944F096
:109FA0008044C2F800490D78D0F83C4805F00F0510
:109FB0000C4E03FA05F5ADB2AC43C0F83C48D0F8FE
:109FC0001C48097801F00F018B4099B28C43C0F80E
:109FD0001C48D2F800093040C2F80009D1E700005F
:109FE0000078F3EF007833ECD0F8001E21F0030185
:109FF000C0F8001ED0F8041821F00201C0F80418BF
:10A0000000207047D0F8001E21F00301C0F8001EA8
:10A01000D0F8041841F00201C0F80418002070477D
:10A020002DE9F04F00250F46904604462E4628465F
:10A0300004EB8001C1F80451401C0F28F8D3C3F38E
:10A0400007405FEA0009204610D0806B40F4001101
:10A05000C4F83810C8F30720C4F8005E0128204671
:10A0600017D0D0F8001841F0030119E0D0F8040827
:10A0700040F00201C4F80418A06B20F40011A163A1
:10A08000206840F040012160206840F0800121609C
:10A09000E0E7D4F80018380E204601D041F0010165
:10A0A000C0F80018102100F08CFA00B101262046FB
:10A0B00000F06BFA00B101264FF67F3A4FF0006CCA
:10A0C000C4F810584FF0904BC4F81458C4F81C58FA
:10A0D0000020FAB214E000BF04EB4011D1F80039BF
:10A0E000002B06DA10B1C1F800B904E0C4F800C9C9
:10A0F00001E0C1F80059C1F81059C1F808A9401C85
:10A100008242E9D8002013E004EB4011D1F8003B73
:10A11000002B06DA10B1C1F800BB04E0C4F800CB94
:10A1200001E0C1F8005BC1F8105BC1F808AB401C4E
:10A130008242E9D8D4F81008C7F30742002A6FF02A
:10A14000804120F48072C4F81028A561616103D1B8
:10A15000A06940F01000A061A069C8F30741094A56
:10A160001043A06119B1A06940F00800A061B9F1E5
:10A17000010F03D1A06904490843A0613046BDE83E
:10A18000F08F000000383C8004000040816821F01E
:10A19000010181600020704710B5144C036CA3428C
:10A1A00003D9D0F8003B002B1EDB0023C0F8103B86
:10A1B0000129D0F8101B41F40021C0F8101BD0F881
:10A1C000101B41F01801C0F8101BD0F8101B41F013
:10A1D000C041C0F8101B07D1C0F8142BD0F8001BE9
:10A1E00041F08021C0F8001B002010BD0A30544F00
:10A1F0000B784A78012A00EB43100BD0D0F8002BE3
:10A2000022F40012C0F8002B0979032914D0022986
:10A2100012D017E0D0F8002922F40012C0F800296B
:10A220000979032901D002290CD1D0F8001941F095
:10A230008051C0F8001905E0D0F8001B41F08051B2
:10A24000C0F8001B002070470A784B78D1B2012B70
:10A2500000EB421012D0D0F8002B002A06DB29B107
:10A26000D0F8001B21F08041C0F8001BD0F8001B83
:10A2700041F40011C0F8001B00207047D0F80029FD
:10A28000002A06DB29B1D0F8001921F08041C0F87E
:10A290000019D0F8001941F40011C0F80019EBE7DB
:10A2A000F8B50B786FF060464F788C4DDCB2012F1B
:10A2B00000EB43132BD0D3F8107B002C07EAC544E6
:10A2C000C3F8104BD3F8104B04EA0504C3F8104B45
:10A2D0007ED00D69002D7CD08C6825446D1EB5FBA9
:10A2E000F4F5ADB26C430C6206EAC545D3F8104BE9
:10A2F0002C43C3F8104BD3F8104B0D6AC5F312056D
:10A3000054EA0504C3F8104B012A73D0CEE00F695C
:10A3100007B3D3F810796FF31207C3F81079D3F8A5
:10A32000107907EA0507C3F810791CB3D1F810C0FB
:10A330008D68D3F81079AC44ACF1010CBCFBF5F599
:10A34000ADB206EAC5463743C3F810790E79012E3F
:10A350001CD02AE0D3F810692E40C3F81069D3F856
:10A36000105945F40025C3F81059D3F810596FF36C
:10A37000120520E00E698D68AE4200D90D61D0F85B
:10A38000106946F40026C0F810690EE0D3F8106991
:10A390004FF0C04707EA457726F0C046C3F810697A
:10A3A000D3F810593D43C3F810590E69D3F810592A
:10A3B000C6F312063543C3F81059012A1BD000EB2F
:10A3C0004413D3F8004944F00444C3F8004901E0C1
:10A3D00047E05AE00C79012C2ED00A695AB30B7869
:10A3E000D0F83418012203F00F039A401143C0F84B
:10A3F000341871E056E0CA691AB100EB4413C3F88F
:10A400001429097901290ED1D0F80818C90500EBE3
:10A410004411D1F8002902D442F0005201E042F088
:10A420008052C1F8002900EB4410D0F8001941F027
:10A430000441C0F800194FE0D0F80848E405D3F80B
:10A44000004902D444F0005401E044F08054C3F8C1
:10A45000004900920B8A0A78C9689BB200F0E0F9C3
:10A460003AE00C690CB18C680C618C680C62C4F326
:10A470001205D0F8104B2C43C0F8104BD0F8104BFD
:10A4800044F40024C0F8104B3EE78D68D3F8104B1D
:10A49000C5F312052C43C3F8104BD3F8104B44F40A
:10A4A00000242FE7CA680AB1C3F8142B09790129DF
:10A4B0000CD1D0F80808C005D3F8000B02D440F046
:10A4C000005001E040F08050C3F8000BD3F8000BBF
:10A4D00040F00440C3F8000B0020F8BDFFFF07E088
:10A4E00038B5002242F21074002300920A784D78A9
:10A4F000012D00EB421219D0D2F8005B002D3CDA9E
:10A50000D2F8005B45F00065C2F8005B0A7800EB0A
:10A510004212D2F8005B45F08045C2F8005B009A19
:10A52000521C0092A24221D9012326E0D2F8005900
:10A53000002D22DAD2F8005945F00065C2F8005922
:10A540000A7800EB4212D2F8005945F08045C2F873
:10A550000059009A521C0092A242E5D80A7800EBFA
:10A560004212D2F80029002AF3DB06E00A7800EB59
:10A570004212D2F8002B002AD1DB184638BD816880
:10A5800041F0010181600020704708B500214FF0C3
:10A5900070620091009B5B1C009393420AD8036990
:10A5A000002BF7DA0091102303610099491C0091F8
:10A5B000914201D9032008BD0169C906F5D40020E4
:10A5C00008BD18B500224FF070630092009C641C17
:10A5D00000949C420CD80469002CF7DA20240092E5
:10A5E00044EA811101610099491C0091994201D905
:10A5F000032018BD01698906F5D4002018BDD0F8E4
:10A60000080810F0060004D0022803D0062801D064
:10A610000F20704702207047406900F0010070472A
:10A62000D0F81818D0F81C08084080B27047D0F84D
:10A630001818D0F81C080840000C704710B5D0F866
:10A64000102801F00F0300EB4114D0F83418D4F8AF
:10A650000809D94001F0010142EAC111084010BDCA
:10A6600000EB4111D1F8081BD0F8140808407047DE
:10A6700041698069084070470346084630B5940830
:10A6800002F00301002203F5805303E01D68521C11
:10A6900040F8045BA242F9D300290CD01C680023C7
:10A6A000491EDD00090403F10103090C24FA05F237
:10A6B00000F8012BF4D130BD70B50446C068012903
:10A6C0004FF0000520F0C040E06001D079B120E0FB
:10A6D000E06840F00050E0600A20F8F7F9F860699F
:10A6E0000A3510F0010F10D1C82DF5D30DE0E06848
:10A6F00040F08040E0600A20F8F7EAF860690A3527
:10A7000010F0010F01D0C82DF5D3C82D01D00020C5
:10A7100070BD012070BDD0F800284FF4FE6303EA3D
:10A72000011322F4FE62C0F80028D0F80018194383
:10A73000C0F8001800207047022A3ED1264A274B55
:10A740000A449A4201D20F2138E0254A254B0A4497
:10A750009A4201D20E2131E0234A244B0A449A4204
:10A7600001D20D212AE0224A224B0A449A4201D208
:10A770000C2123E0204B214A0B44934201D20B21B0
:10A780001CE01F4B1F4A0B44934201D20A2115E0E3
:10A790001D4B1E4A0B4493420FD31D4B1D4A0B44C5
:10A7A000934201D2082109E01B4B1C4A19449142F3
:10A7B00001D2072102E0062100E00921C2684FF41E
:10A7C000705322F47052C26003EA8123C1681943B6
:10A7D000C160002070470000405327FF00350C0087
:10A7E000401E1BFF40420F0000DC0BFF804F120099
:10A7F000808CF9FE20D6130060B6E5FE60E31600FB
:10A8000000D3CEFE40771B00C05BB3FEC091210099
:10A8100000CA91FE20753800E05459FEE09C4100CA
:10A8200010B5029C74B900EB0232DB1C00209B08BF
:10A8300002F5805204E000BF51F8044B1460401C44
:10A840009842F9D3002010BDFEE7090700284FEA1F
:10A85000116104DB00F1E02080F80014704700F083
:10A860000F0000F1E02080F8141D7047F8F70EFD8E
:10A87000FDF72EFCFCF7C8FDFCF706FDFCF7AAFC73
:10A88000FCF754FFFCF7BEFEFCF71EFFFCF7EAFEE8
:10A89000FDF728F8FDF7C8F8FDF7FAF8FDF72EF9EF
:10A8A000FDF75AF8FDF78CF8FCF704FDFCF734FDD2
:10A8B000FCF766FDFCF774FFFCF7D2FFFCF768FEBF
:10A8C00000F014F8FCF790FD00F022F8FEE710B558
:10A8D000EFF3058111B16FF0050404E04FF00004BF
:10A8E00008B100F001FE204610BD0000EFF3058026
:10A8F00010B16FF0050070470449086810B14FF0BF
:10A90000FF30704701220A60002070475800002085
:10A9100010B5EFF3058010B16FF0050010BD0848C9
:10A920000168012902D04FF0FF3010BD054A002117
:10A9300082F8141D0221016000F03EFE002010BDCF
:10A94000580000200BE000E02DE9FF414FEA010331
:10A950004FF00005EFF30581039561BB58B34FF04D
:10A9600080064FF018014FF000044AB3176807B192
:10A970003C4697691FB139467F1E382F02D217799E
:10A98000FF0703D0002004B0BDE8F081576907B18C
:10A99000BE08D2F808C0BCF1000F0DD0D5685C2D00
:10A9A00018D312693AB137B18DE806103246214604
:10A9B00001F0A5F903900DE0D7685FB912694AB9B3
:10A9C00003AACDE90012B2B2214601F06BF90128C9
:10A9D00000D003950398D6E72DE9F041134C0F46BC
:10A9E0000546E6682068001D00F048FC681C07D199
:10A9F00037B12168BDE8F0410D48091D00F090BC59
:10AA000020683544B5424560216805D2A06B091D18
:10AA1000BDE8F04100F06CBC606B091D00F068FC03
:10AA2000A06A854200D2A562BDE8F0814C000024F6
:10AA3000A41100242DE9F041054600F07DFC2D4CC9
:10AA40002D4FA068401CA060206810B1606930B331
:10AA50002BE02560A068012827D1002606EB8600A0
:10AA600007EB800000F036FC761C382EF6D3234826
:10AA700000F030FC2148143000F02CFC1F48283036
:10AA800000F028FC1D483C3000F024FC1B485030EE
:10AA900000F020FC194860631430A06305E0E86A08
:10AAA0002168C96A814200D82560606A401C6062E2
:10AAB0006864E86A2169884200D9206100EB80005F
:10AAC000291D07EB800000F02BFC00F055FC6069AD
:10AAD00000280CD02068E96AC06A884207D2084979
:10AAE0004FF080500860BFF34F8FBFF36F8FBDE80A
:10AAF000F08100004C000024F40C002454110024C8
:10AB000004ED00E038B500F017FC104C2068C8B91F
:10AB10000F4800F0DFFB0E48143000F0DBFB0C495F
:10AB20000020E16014312161A1F582730090A1F150
:10AB3000B40210210A2000F04DFE206010B105A1E2
:10AB400000F09CFCBDE8384000F016BC440000203A
:10AB5000A8120024546D72510000000030B4026C41
:10AB60000B46002A0BD0D0E902411144C160A1423A
:10AB700001D30168C160184630BCF5F720BD30BC78
:10AB800070472DE9F041856B1746026C044600269C
:10AB900082B1C7B1E068F5F712FDE168206C226868
:10ABA000091AE160914202D2A168081AE060022FFE
:10ABB00016D017E02068A8B9A06801F043F906464E
:10ABC0000020A0600EE06068F5F7F9FCD4E901010F
:10ABD000226C10446060884204D32068606001E009
:10ABE00005B16D1E6D1CA5633046BDE8F08110B542
:10ABF000044690F8590058B101280CD002280FD013
:10AC0000502080F31188BFF34F8FBFF36F8FFEE7A3
:10AC1000206B00F0C5FB2046BDE8104000F0C0BB33
:10AC200010BD000011484FF4C04110B5420706D0D6
:10AC30000E49C01D20F00700411AC1F5C0410C4C5F
:10AC4000002301440839A4F1180221F00701C4E9E6
:10AC500000030C1A11604B600B60C0E90014946093
:10AC60004FF000415460516110BD0000E819002010
:10AC700074000020144E4FF08058144CDFF85090B0
:10AC8000A6F29C4712E000BF00F056FBF068C568D2
:10AC9000281D00F0F3FAA068401EA0606068401E06
:10ACA000606000F069FB2846FFF7A1FF606800289C
:10ACB000EAD138680128F9D9C9F80080BFF34F8F6D
:10ACC000BFF36F8FF2E70000901100244C000024C6
:10ACD00004ED00E070B51D46049C51B1C4F800209D
:10ACE000C4E90F010121204600F0A8FD84F84C5072
:10ACF00070BD2460F4E72DE9F05F88469A46910024
:10AD00001546DDE90B940A9EA5228346206BF5F7D4
:10AD1000CDFC206B6FF0030101EB8501084420F0AE
:10AD20000707780707D0502080F31188BFF34F8FB3
:10AD3000BFF36F8FFEE7B8F1000F4FF000050ED0A4
:10AD40000020221818F8001082F8341018F80010AB
:10AD500011B1401C1028F4D384F8435001E084F86A
:10AD60003450382E00D33726E662201DC4E913651F
:10AD700000F0BBFA04F1180000F0B7FA6565C6F1FF
:10AD80003800A06184F8585052462461594638462C
:10AD9000646200F05BFAB9F1000F206001D0C9F8DD
:10ADA0000040BDE8F09F000030B5114900E01146B9
:10ADB0000A688242FBD34B685C18844203D1446822
:10ADC000084623444B6043681D18954209D1084C3E
:10ADD000183C2468A24209D052681A4442600A68AA
:10ADE00012680260814200D0086030BD0460F9E75B
:10ADF0007400002070B50D4D914241604FF0000489
:10AE0000006106D88169D21A8A4206D2011D2869DA
:10AE100007E09A4203D2994201D3012403E0011DC5
:10AE2000E86800F065FA204670BD0000440000208C
:10AE300010B5044600F080FAA06B28B15FF0000462
:10AE400000F09AFA204610BD0124F9E730B53C4DD8
:10AE500089B06BE00498002806DA059ADDE906015E
:10AE600090470498002861DB069C606910B1201DA2
:10AE700000F004FA03A800F0D5F8024604980A2866
:10AE800054D2DFE800F00505052D304705052D30CB
:10AE900094F8280040F0010084F82800A069059982
:10AEA0000B4601442046FFF7A5FF50B3216A204618
:10AEB000884794F82800400738D50020009005986E
:10AEC0000023A16942181946204601F0C3F8C0B911
:10AED000502080F31188BFF34F8FBFF36F8FFEE7D1
:10AEE00094F828001EE094F8280040F0010084F84F
:10AEF00028000598A06128B1811813462046FFF765
:10AF000079FF13E0502080F31188BFF34F8FBFF318
:10AF10006F8FFEE794F82800810703D4204600F0E5
:10AF20003FFA03E020F0010084F82800286800229E
:10AF300004A900F0DDFD00288CD109B030BD00006F
:10AF4000440000202DE9FC410F46054600F078FB47
:10AF500001A800F067F80446019818B100F0E8FF76
:10AF6000BDE8FC81254EAFB130690068D0B3002741
:10AF70003068291B3A4600F095FA00F0D9FF002806
:10AF8000EED11F494FF080500860BFF34F8FBFF3E1
:10AF90006F8FE5E7A542EBD800F0CAFFF0682746BF
:10AFA000C068C468201D00F069F994F828004107C2
:10AFB00019D5A0692B463A4641192046FFF71AFFDA
:10AFC000A8B100202A46034601460090204601F021
:10AFD00041F860B9502080F31188BFF34F8FBFF361
:10AFE0006F8FFEE707E020F0010084F82800216A57
:10AFF00020468847B4E70127BAE700004400002054
:10B0000004ED00E00648416B096829B1416BC9684D
:10B01000C9684968816270474FF0FF31FAE7000064
:10B020004C00002470B5054600F0A2FE064E044612
:10B03000B068844203D200F009F8012000E000204B
:10B0400028602046B46070BD44000020F8B5194D5A
:10B0500020E0C068C4680668201D00F00FF9216A6E
:10B060002046884794F82800400713D5A06930444B
:10B07000B04206D92461211D6060E86800F038F90B
:10B0800008E000203246034601460090204600F0CA
:10B09000E1FF38B1E86801680029DAD12969C5E91A
:10B0A0000310F8BD502080F31188BFF34F8FBFF31A
:10B0B0006F8FFEE74400002008484068401C4FF0B6
:10B0C000500080F3118804D0BFF34F8FBFF36F8F10
:10B0D000FEE7BFF34F8FBFF36F8FFEE77C000020CA
:10B0E000074CE068016841B1C0680021D0F8000059
:10B0F000FFF728FFFFF7AAFEF3E701210020F7E79B
:10B10000440000202DE9F041044600F015F994F9BF
:10B11000455004F1240609E0606A48B1304600F069
:10B12000CFFE08B100F00EFA6D1E6DB2002DF3DCFB
:10B130004FF0FF3684F8456000F01EF900F0FCF88F
:10B1400094F9445004F1100709E0206948B13846E9
:10B1500000F0B6FE08B100F0F5F96D1E6DB2002DDD
:10B16000F3DC84F84460BDE8F04100F005B900006C
:10B170002DE9F0410027044600F062FA324E3068B3
:10B1800008B9FFF74FFD706904424ED1C4B30834CB
:10B1900060070ED004F00700C0F108000444600707
:10B1A00007D0502080F31188BFF34F8FBFF36F8F0C
:10B1B000FEE72CB37068844237D823481830014624
:10B1C0000D6801E028460D466968A14202D229684F
:10B1D0000029F7D131688D4227D0076829680160BE
:10B1E00008376868011B10290FD92819420708D0B1
:10B1F000502080F31188BFF34F8FBFF36F8FFEE7AE
:10B2000013E041606C60FFF7CFFD69687068401A19
:10B210007060B268904200D2B06000207269114341
:10B22000C5E90001F068401CF06000F081FE78077D
:10B2300007D0502080F31188BFF34F8FBFF36F8F7B
:10B24000FEE73846BDE8F0815C00002070B5041FC1
:10B25000094E231F4FF0807521F0010125601C1F4E
:10B260001960A0F120010B1F266044380A606FF0BE
:10B2700002051D6070BD0000B9B00008D0E90132C0
:10B2800001699A60D0E901235A604A68824201D17B
:10B2900082684A60002202610868401E08600868EF
:10B2A0007047000010B5044C8023046004F15C007A
:10B2B0000860136010BD0000D012002410B5044CCB
:10B2C0004FF48073046004F15C000860136010BDEB
:10B2D0002C1500244FF0FF3300F108010022C0E9D3
:10B2E00001130260C1600161704700210161704774
:10B2F00030B50B685A1C02D000F1080202E0026966
:10B3000004E02246546825689D42FAD953684B6090
:10B3100099608A60516008610168491C016030BD14
:10B3200042684A6093688B609368596091600861D5
:10B330000168491C01607047502080F31188BFF3F9
:10B340004F8FBFF36F8F0A494868401C486001283F
:10B350000CD10848006810F0FF0F07D0502080F390
:10B360001188BFF34F8FBFF36F8FFEE77047000068
:10B370007C00002004ED00E00849486828B1401E28
:10B38000486001D180F311887047502080F3118804
:10B39000BFF34F8FBFF36F8FFEE700007C000020EC
:10B3A00070B500282AD0164DA0F1080461686869BC
:10B3B000014207D1502080F31188BFF34F8FBFF3B4
:10B3C0006F8FFEE722683AB1502080F31188BFF3F7
:10B3D0004F8FBFF36F8FFEE78143616000F030F95C
:10B3E00060686968084468602046FFF7DDFC2869EA
:10B3F000401C2861BDE8704000F09ABD70BD00009F
:10B400005C0000204FF0E020002101614FF47A72CF
:10B410008161072303490968B1FBF2F1491E4161CB
:10B42000036170474400002410B5F5F729F811496D
:10B4300010280ED300F1E0200A7890F8F003904233
:10B4400007D2502080F31188BFF34F8FBFF36F8F67
:10B45000FEE709488968006800F4E060884207D97F
:10B46000502080F31188BFF34F8FBFF36F8FFEE73B
:10B4700010BD00007C0000200CED00E0084B5FF0E8
:10B48000000210B553F832401CB1521C082AF9D3FF
:10B4900010BD03EBC20443F83210606010BD000021
:10B4A000B40C002470B515460E460446FFF744FF61
:10B4B00094F944100020491C01D184F8440094F907
:10B4C0004510491C01D184F84500FFF755FFA06BDA
:10B4D00028B904F124002A46314600F051F82046EC
:10B4E000BDE87040FFF70EBE020010B514D00F4843
:10B4F000006B38B1502080F31188BFF34F8FBFF33A
:10B500006F8FFEE700F09CF800211046FFF764FA09
:10B5100000F00EFD002807D105494FF0805008606B
:10B52000BFF34F8FBFF36F8F10BD00004C0000249E
:10B5300004ED00E002490A6A0260C9684160704790
:10B540004C00002401490120C86170474C000024D0
:10B5500010B50C4650B1094909681831FFF7C8FE0B
:10B560002046BDE810400121FFF736BA502080F395
:10B570001188BFF34F8FBFF36F8FFEE74C0000249D
:10B5800070B514460D4668B10A4909681831FFF7CD
:10B59000C7FE0CB14FF0FF3521462846BDE870408C
:10B5A000FFF71ABA502080F31188BFF34F8FBFF313
:10B5B0006F8FFEE74C00002430B587B0002405AA49
:10B5C00004A9039403A80494FFF76CFEDDE90301CA
:10B5D00000940023CDE90110174815A1059A00F049
:10B5E0008EFB164D0028E8621FD000F003FD0128F5
:10B5F00009D0401C19D1502080F31188BFF34F8F20
:10B60000BFF36F8FFEE7502080F31188BFF34F8F99
:10B61000BFF36F8F01214FF0FF30A8626961EC60CA
:10B6200007B0BDE8304000F045B807B030BD0000BD
:10B6300049444C450000000075AC00084C00002453
:10B640000248016B491C0163704700004C00002454
:10B65000164810B5016B11B10121C16110BD002167
:10B66000C161134A016901E0B9B1491E01EB8103CF
:10B6700052F82330002BF7D001EB810302EB830259
:10B6800002F1080453685B685360A34201D15B6810
:10B690005360DA680260016110BD502080F31188A8
:10B6A000BFF34F8FBFF36F8FFEE700004C00002405
:10B6B000F40C002437481CB5374902688A4207D188
:10B6C000502080F31188BFF34F8FBFF36F8FFEE7D9
:10B6D00031490068491E884207D1502080F3118803
:10B6E000BFF34F8FBFF36F8FFEE72C49FF200A781F
:10B6F0000192087008788DF800009DF800209DF8F0
:10B70000000002F0F002824207D0502080F311883E
:10B71000BFF34F8FBFF36F8FFEE79DF80020072028
:10B720001F4C02F050022270A06005E09DF800203E
:10B7300052008DF80020401E9DF800201206F5D41E
:10B740000328A06007D0502080F31188BFF34F8FEB
:10B75000BFF36F8FFEE74FF44070A0600198087050
:10B760000C482030016841F470010160016841F02B
:10B7700070410160FFF746FE00206060F4F748FE6C
:10B780000848016841F040410160F4F72DFE0020B7
:10B790001CBD000000ED00E071C20F4100E400E0BC
:10B7A0007C00002034EF00E0502010B580F31188B9
:10B7B000BFF34F8FBFF36F8F00F0E0FA18B1044969
:10B7C0004FF080500860002080F3118810BD000009
:10B7D00004ED00E0F8B5069D18B153B1CAB181B1CE
:10B7E00020E0502080F31188BFF34F8FBFF36F8F9D
:10B7F000FEE7502080F31188BFF34F8FBFF36F8FA8
:10B80000FEE7502080F31188BFF34F8FBFF36F8F97
:10B81000FEE739B1502080F31188BFF34F8FBFF39B
:10B820006F8FFEE750241C46012683F84660009384
:10B830002B46FFF74FFA2046F8BD00002DE9F047F0
:10B8400004008A4629D0FFF777FD21680025D4E956
:10B850000F23D4F840C004F1100810460E46401ED5
:10B860004FF0FF3902FB031200FB0C10BAF1000F7E
:10B87000A563666084F8449084F84590C4E902208A
:10B8800013D04046FFF726FD04F12400FFF722FD08
:10B89000FFF772FD0120BDE8F087502080F311888A
:10B8A000BFF34F8FBFF36F8FFEE720690028EFD003
:10B8B000404600F005FB0028EAD004494FF08050D4
:10B8C0000860BFF34F8FBFF36F8FE1E704ED00E037
:10B8D0002DE9FF4704001D4682B08A464FF000085C
:10B8E00003D0BAF1000F08D011E0502080F3118886
:10B8F000BFF34F8FBFF36F8FFEE7206C38B150203E
:10B9000080F31188BFF34F8FBFF36F8FFEE7022DD7
:10B910000AD1E06B012807D0502080F31188BFF3D3
:10B920004F8FBFF36F8FFEE700F014FA3F4F4FF0D9
:10B9300080564FF0000948B9049838B1502080F380
:10B940001188BFF34F8FBFF36F8FFEE7FFF7F4FC53
:10B95000A06BE16B884207D3022D05D00498D0B1CB
:10B96000B8F1000F1AD01EE02A4651462046FFF7D4
:10B9700008F9616A19B104F1240000F0A1FA20B1BC
:10B980003E60BFF34F8FBFF36F8FFFF7F5FC0120D1
:10B9900006B0BDE8F087FFF7EFFC22E06846FFF74E
:10B9A000C9FD4FF00108FFF7E7FCFFF749FEFFF77D
:10B9B000C3FC94F94400401C01D184F8449094F9EC
:10B9C0004500401C01D184F84590FFF7D5FC04A93F
:10B9D000684600F02BF930B12046FFF793FB00F0EA
:10B9E000A7FA0020D4E7FFF7A7FCA06BE16B884221
:10B9F00013D1FFF7C1FC049904F11000FFF7A8FD73
:10BA00002046FFF77FFB00F093FA00289ED13E60AE
:10BA1000BFF34F8FBFF36F8F98E7FFF7ADFC204662
:10BA2000FFF770FB00F084FA90E7000004ED00E0FF
:10BA30002DE9F04704001F469046894603D0B9F12E
:10BA4000000F08D011E0502080F31188BFF34F8F12
:10BA5000BFF36F8FFEE7206C38B1502080F3118860
:10BA6000BFF34F8FBFF36F8FFEE7022F0AD1E06B5A
:10BA7000012807D0502080F31188BFF34F8FBFF308
:10BA80006F8FFEE7FFF7D0FC5020EFF3118680F3B5
:10BA90001188BFF34F8FBFF36F8FA06BE16B8842AC
:10BAA00006D3022F04D0002086F31188BDE8F0876A
:10BAB00094F94550A06B3A4649462046FFF761F895
:10BAC000681C04D06D1C84F845500120ECE7606AC6
:10BAD0000028FAD004F1240000F0F2F90028F4D094
:10BAE000B8F1000FF1D00121C8F80010EDE7000017
:10BAF0002DE9F74704008A4683B04FF0000603D0D3
:10BB0000BAF1000F08D011E0502080F31188BFF384
:10BB10004F8FBFF36F8FFEE7206C38B1502080F35A
:10BB20001188BFF34F8FBFF36F8FFEE700F012F95C
:10BB3000DFF8F4804FF080574FF0000948B90598BE
:10BB400038B1502080F31188BFF34F8FBFF36F8F50
:10BB5000FEE7FFF7F1FBA56BC5B151462046FEF7A6
:10BB6000FDFF6D1EA563206950B104F1100000F0C7
:10BB7000A7F928B1C8F80070BFF34F8FBFF36F8FDC
:10BB8000FFF7FAFB012006B0BDE8F087059808B181
:10BB90001EB106E0FFF7F0FB27E06846FFF7CAFC9E
:10BBA0000126FFF7E9FBFFF74BFDFFF7C5FB94F913
:10BBB0004400401C01D184F8449094F94500401C95
:10BBC00001D184F84590FFF7D7FB05A9684600F03E
:10BBD0002DF8002820460AD0FFF794FA00F0A8F9C3
:10BBE0002046FFF725F90028B3D00020CBE7FFF768
:10BBF0001FF990B1059904F12400FFF7A9FC204634
:10BC0000FFF780FA00F094F90028A2D1C8F800707C
:10BC1000BFF34F8FBFF36F8F9BE72046FFF772FA9A
:10BC200000F086F995E7000004ED00E02DE9F04111
:10BC300005000C4612D0CCB1FFF77EFB184E2068F1
:10BC4000F268471C6B68A2EB030117D02F68366AB5
:10BC5000B74215D0934213D801251CE0502080F341
:10BC60001188BFF34F8FBFF36F8FFEE7502080F333
:10BC70001188BFF34F8FBFF36F8FFEE700250AE0F7
:10BC8000884205D9401A20602846FFF753FCF5E7A3
:10BC9000002020600125FFF76FFB2846BDE8F081FA
:10BCA0004C0000242DE9FF5F994616468A468346DC
:10BCB0009000DDE90E87FFF75BFA05001CD05C20E1
:10BCC000FFF756FA040014D00020256384F85900C9
:10BCD0004B46CDE90087CDE90240324651465846F1
:10BCE000FFF709F82046FEF7A5FE012004B0BDE8E5
:10BCF000F09F2846FFF754FB4FF0FF30F6E7F0B512
:10BD000085B0DDE90B740A9DA7B1DCB15C26276321
:10BD1000022684F85960002703970DF1100C009556
:10BD2000CDE901C4FEF7E7FF2046FEF783FE049845
:10BD300005B0F0BD502080F31188BFF34F8FBFF3E3
:10BD40006F8FFEE7502080F31188BFF34F8FBFF352
:10BD50006F8FFEE70548416919B1006B18B10020EB
:10BD60007047012070470220704700004C000024FB
:10BD70000148C068704700004C0000242DE9F041E4
:10BD80002E4C206B002728B1A069401CA0613846CA
:10BD9000BDE8F081E668761CE66013D1606B006850
:10BDA00038B1502080F31188BFF34F8FBFF36F8FEE
:10BDB000FEE7606BA16B6163A063206A401C206298
:10BDC000FFF720F9DFF87880A06A864209D3606B1C
:10BDD0000068A0B1606BC068C5686868864211D20F
:10BDE000A0622068C06A00EB800158F82100012899
:10BDF00000D90127E0690028C9D00127C7E74FF023
:10BE0000FF30EDE7281DFFF739FAA86A18B105F1F0
:10BE10001800FFF733FAE86A2169884200D92061E7
:10BE200000EB800108EB8100291DFFF779FA2068FB
:10BE3000E96AC06A8142CAD30127C8E74C000024DE
:10BE4000F40C002470B504464FF0000190B31A4D75
:10BE50002868844207D0502080F31188BFF34F8FA9
:10BE6000BFF36F8FFEE7206D38B1E36C401EE26ACE
:10BE700020659A421ED040B11CE0502080F311880A
:10BE8000BFF34F8FBFF36F8FFEE7201DFFF7F6F96B
:10BE9000E06CC0F13801A161E0622969884200D9F3
:10BEA000286100EB8000054901EB8000211DFFF7B0
:10BEB00037FA0121084670BD4C000024F40C002420
:10BEC00070B5C068C46854B104F118000646FFF7A5
:10BED000D5F9144D286B50B11348314615E0502068
:10BEE00080F31188BFF34F8FBFF36F8FFEE7201DE4
:10BEF000FFF7C4F9E06A2969884200D9286100EB9C
:10BF000080000A4901EB8000211DFFF709FAE06A71
:10BF10002968C96A884203D90121E961084670BDD0
:10BF2000002070BD4C0000247C110024F40C00247F
:10BF30002DE9F0472C4D286B0024274638B1FFF738
:10BF4000FBF9286B401E2863286B40B147E0502066
:10BF500080F31188BFF34F8FBFF36F8FFEE7234E3F
:10BF60000120A968D9B3A6F5916980463068E0B18F
:10BF7000F068C46804F11800FFF780F9201DFFF78E
:10BF80007DF9E06A2969884200D9286100EB8001C7
:10BF900009EB8100211DFFF7C3F9E06A2968C96A2E
:10BFA0008842E3D3C5F81C80E0E70CB1FFF72AF81C
:10BFB000AC694CB14FEA0806FFF7E0FE00B1EE6154
:10BFC000641EF9D10020A861E86940B10849012741
:10BFD0004FF080500860BFF34F8FBFF36F8FFFF7B4
:10BFE000CBF93846BDE8F0874C0000247C110024D2
:10BFF00004ED00E010B586B0FEF784FD114C20681A
:10C00000B8B10020039005AA049004A903A8FFF783
:10C0100055F9DDE90321022000238DE807000C48D3
:10C0200009A1059AFFF76BFE606010B106B0012010
:10C0300010BD502080F31188BFF34F8FBFF36F8F77
:10C04000FEE7000044000020546D72205376630028
:10C05000E1B000082DE9FF411E46134602004FF0F3
:10C0600000000A9D16D0144C2768002F0FD0062917
:10C070000292CDE9001317DAFFF76CFE02284FF0A9
:10C0800000030FD0002220686946FFF721FC04B0AE
:10C09000BDE8F081502080F31188BFF34F8FBFF3CC
:10C0A0006F8FFEE72A46EEE70023324669463846A0
:10C0B000FFF7BEFCEBE70000440000204FF04070AB
:10C0C000E1EE100A7047000088C10008000000007F
:10C0D000000000000000000000000000000200005E
:10C0E000180000000000000000000000000610160C
:10C0F000000610160001020304050607080C1014C0
:10C100001820304000000000000000000000000087
:10C11000000000000000000001000000020000001C
:10C120000300000004000000000000000500000003
:10C1300000000000000000000000000006000000F9
:10C1400000000000000000000000000007000000E8
:10C15000010002000400060008000A000C001000A4
:10C1600020004000800000010101010307010000E0
:10C170000804020408010101000000000102030498
:10C18000010203040607080964656661756C74544E
:10C1900061736B00D4C1000800000020C0000000E3
:10C1A0006403000894C2000800000024E0000000BE
:10C1B0006403000894C20008C00000202879000031
:10C1C0008003000874C30008E00000240879000020
:10C1D00080030008000000000403090412010002AB
:10C1E00002020040830440570002010203010000E4
:10C1F000050F0C0001071002020000001A030000E6
:10C20000000000000000000000000000000000002E
:10C21000000000000000000000000000000000001E
:10C22000000000000000000000000000000000000E
:10C2300000000000000000000000000000000000FE
:10C2400000000000000000000000000000000000EE
:10C2500000000000AAAAAAAA00000000818F00081E
:10C26000ED8D000823910008000000007D8E00087D
:10C27000398D0008AF8D00080000000000000000AC
:10C2800000000000018F0008C18E0008418F0008E7
:10C29000B58E00080000000085940008B5940008E1
:10C2A000C1940008E99400081595000865940008F9
:10C2B0009194000800000000B9080008B3080008C5
:10C2C000AF080008DD080008F508000801000000BC
:10C2D00010000000000000000090D0030090D00388
:10C2E000000000000000000000000000000000004E
:10C2F000000000000000000000000000000000003E
:10C30000000000000000000000000000000000002D
:10C31000000000000000000000000000000000001D
:10C32000810182000A0600020000004001000000B6
:10C3300009024300020100C03209040000010202A8
:10C34000010005240010010524010001042402025B
:10C3500005240600010705820308001009040100F6
:10C36000020A0000000705010240000007058102E3
:04C370004000000089
:04000005080002CD20
:00000001FF
